:020000040000FA
:10000000302D0020F902000001030000030300006E
:1000100005030000070300000903000000000000C2
:100020000000000000000000000000000B030000C2
:100030000D030000000000000F030000110300008A
:100040001303000039070000F90A00001303000041
:1000500013030000130300009504000013030000C5
:10006000950A0000130300001303000013030000AF
:100070001303000013030000130300001303000028
:1000800013030000C907000013030000130300005E
:10009000ED070000F1070000130300001303000048
:1000A00013030000130300001303000013030000F8
:1000B0001303000013030000000000000000000014
:1000C00013030000130300001303000013030000D8
:1000D00013030000130300001303000013030000C8
:1000E00013030000130300001303000000000000CE
:1000F00000000000130300000000000013030000D4
:1001000000000000000000000000000000000000EF
:1001100000000000000000000000000000000000DF
:1001200000000000000000000000000000000000CF
:1001300000000000000000000000000000000000BF
:1001400000000000000000000000000000000000AF
:10015000000000000000000000000000000000009F
:10016000000000000000000000000000000000008F
:10017000000000000000000000000000000000007F
:10018000000000000000000000000000000000006F
:10019000000000000000000000000000000000005F
:1001A000000000000000000000000000000000004F
:1001B000000000000000000000000000000000003F
:1001C000000000000000000000000000000000002F
:1001D000000000000000000000000000000000001F
:1001E000000000000000000000000000000000000F
:1001F00000000000000000000000000000000000FF
:10020000DFF80CD000F016F900480047B5300000C8
:10021000302D002030B4044654E8000F0D4644E869
:100220000053002BF8D1156030BC704730B4044641
:1002300054E8000F40EA010544E80053002BF7D1D1
:10024000156030BC704730B4044654E8000F00EA33
:10025000010544E80053002BF7D1156030BC70470E
:1002600030B4044654E8000F80EA010544E8005326
:10027000002BF7D1156030BC704730B4044654E809
:10028000000F00EB010544E80053002BF7D1156087
:1002900030BC704730B4044654E8000FA0EB0105B1
:1002A00044E80053002BF7D1156030BC704770B4A0
:1002B00004464FF0000054E8006F0D68AE4207BFDF
:1002C00044E80023012044E800630E60002B1CBFBB
:1002D0000020F0E770BC704730B4044654E8000FCB
:1002E00088422CBF451A054644E80053002BF5D13F
:1002F000156030BC7047000006488047064800473C
:10030000FEE7FEE7FEE7FEE7FEE7FEE7FEE7FEE7C5
:10031000FEE7FEE765080000010200002DE9F05F3E
:100320000546002092469B46884606468146402464
:100330001BE0284641464746224600F06BF85346EC
:100340005A46C01A914110D311461846224600F071
:1003500016F82D1A67EB01084F46224601200021AE
:1003600000F00DF817EB00094E41201EA4F1010426
:10037000DFDC484631462A464346BDE8F09F202A46
:1003800004DB203A00FA02F1002070479140C2F1EC
:10039000200320FA03F31943904070470048704748
:1003A0005C7C000040EA01039B0703D009E008C918
:1003B000121F08C0042AFAD203E011F8013B00F82A
:1003C000013B521EF9D27047D2B201E000F8012B76
:1003D000491EFBD270470022F6E710B513460A46C5
:1003E00004461946FFF7F0FF204610BD421C10F8E6
:1003F000011B0029FBD1801A704730B5044600204C
:10040000034600E05B1C934203D2E05CCD5C401BE2
:10041000F8D030BD202A04DB203A21FA02F0002176
:10042000704721FA02F3D040C2F120029140084304
:1004300019467047064C074D06E0E06840F001039E
:1004400094E8070098471034AC42F6D3FFF7DCFE7F
:10045000FC7C00001C7D000030B58C1810F8012BCE
:1004600012F00F0301D110F8013B120906D110F868
:10047000012B03E010F8015B01F8015B5B1EF9D171
:1004800001E001F8013B521EFBD1A142E6D300205E
:1004900030BD00002DE9F04F00268DB0DFF8A081BF
:1004A000B14604964FF480750124374605962846D8
:1004B00003F092FD38B1D8F80403204203D0284657
:1004C00003F080FD26432D1D64007F1CADB2082F74
:1004D000EDD34FF4BE74204603F07EFD48B12046B4
:1004E00003F070FD46F0004604AA0221002003F04C
:1004F00053FD544C16F0FF0F15D00127002537424D
:100500000DD008EB8501D1F81005D1F81015C0F316
:10051000052054F82520C1F3014102B190477F0026
:100520006D1C082DEBD3002E7EDA0020CDF828902C
:10053000411E0DF1100B07AACDF82C9042F82010A7
:10054000401C91460228F9D300252E46A11911F826
:10055000607F91F9000027F0C008401C40D007A937
:10056000404602F0CBFF40B34FEA971A404601F0F5
:1005700039FF54F820701FB1BAF1030F03D006E021
:10058000BAF1030F2CD10AA9404602F0BFFF02A81E
:10059000CDF8088003F0A4FC029900EB8100D0F8AC
:1005A000000704A9C0F301400290404602F0A6FFF4
:1005B0000028029802D0022802D011E003280FD1AF
:1005C000BAF1030F08D10298022833D00221404625
:1005D00003F060FC6D1CEDB217B151464046B847C0
:1005E000761C042EB2D3002D21D001AA02210020B6
:1005F00003F0D2FC00205A460DF1040152F82060AD
:1006000051F82030B34217D000200AAE4FEA090358
:1006100051F8207042F8207056F8207043F820708E
:10062000401C0228F4D300E001E0002D8CD10DB075
:10063000BDE8F08F0321CAE7401C0228DED3F6E7AD
:10064000006000402002002000F01F0201219140C4
:100650004009800000F1E020C0F88012704700F0EF
:100660001F02012191404009800000F1E020C0F804
:100670008012704700F01F02012191404009800064
:1006800000F1E020C0F88012704700F01F02012145
:1006900091404009800000F1E020C0F880127047CE
:1006A00000F01F02012191404009800000F1E0208C
:1006B000C0F88011704700F01F02012191404009ED
:1006C000800000F1E020C0F80011704700F01F0228
:1006D000012191404009800000F1E020C0F80011A4
:1006E000704700F01F02012191404009800000F195
:1006F000E020C0F8001270474907090E002806DA0A
:1007000000F00F0000F1E02080F8141D704700F1A8
:10071000E02080F8001470474907090E002806DA27
:1007200000F00F0000F1E02080F8141D704700F188
:10073000E02080F80014704770B5204D28696C786F
:10074000401C2861687D10B11D4802F067FE2878C2
:1007500003281AD11B48D0F80C01B0B1012C04D0E9
:10076000022C0AD01648123023E02869032816D03C
:100770001348083002F052FE11E02869022812D016
:100780000F480D3002F04AFE0DE0032C0FD2012C71
:1007900005D0022C07D0BDE8704004F081BEBDE852
:1007A000704004F0A9BEBDE8704005F0BBB8044835
:1007B0002830BDE8704002F031BE0000E40900209E
:1007C00038030A000010004007480021C0F840111B
:1007D000C0F84411C0F84811C0F84C11C0F800111D
:1007E000C0F8041106F052BF0010014006F0A0BE90
:1007F00030B51B4C85B00025012080F31088D4F85B
:10080000D40038B3D4F8D00000EB800004EB8000B3
:1008100001798DF800108168C26803694069CDE9EB
:100820000330CDE90112D4F8D400401EC4F8D4003E
:10083000D4F8D000401CC4F8D000D4F8D0000A2866
:1008400001D3C4F8D050002080F310882168684696
:100850008847D1E7002080F3108805B030BD000044
:10086000000A002030B54FF0805000228300D0F8FD
:100870003011C3F80C21C3F81021624B1A60624B8F
:100880001B68624C2360604B1B1D1B68241D23608A
:100890005D4B08331B68241D23605B4B0C331B68C6
:1008A000241D2360584B10331B68241D2360564BB6
:1008B00014331B68241D2360534B18331B68534C9F
:1008C00020342360504B1C331B68241D23604E4B87
:1008D00020331B68241D23604B4B24331B68241DCD
:1008E0002360494B28331B68241D2360464B2C335F
:1008F0001B68241D2360444B30331B68434C403439
:100900002360414B34331B68241D23603E4B383336
:100910001B68241D23603C4B3C331B68241D236053
:10092000394B40331B68241D23600124082902D160
:10093000D0F8343113B1082904D006E0354B3449DE
:10094000196005E0D0F8343113B1082904D006E06D
:10095000314BFB21196005E0D0F8343113B108297F
:1009600008D00EE090F858322C48016863F3030178
:10097000016002E0D0F834311BB929494FF400700E
:10098000086028480168C90702D06FF001010160C2
:100990002548016841F470010160BFF34F8FBFF338
:1009A0006F8F4FF01021D1F80002002803DBD1F83F
:1009B0000402002822DA1D4B1C601D480468002C2C
:1009C000FCD01224C1F800420568002DFCD0C1F80B
:1009D000044201680029FCD01A6001680029FCD09B
:1009E000BFF34F8F10487C380168124A01F4E06170
:1009F00011430160BFF34F8F00BFFDE70F490E4861
:100A0000086030BD380500400404001020C50040D7
:100A1000488103008C56004018F50040E40E004069
:100A2000409602400004004088ED00E004E50140EB
:100A300000E401400400FA050090D003F800002013
:100A4000124A10B50021104B126809E053F82140FA
:100A5000844203D10E4802F0E1FC13E0491CC9B204
:100A60009142F3D3084A002112F1180201EB01135D
:100A700002EB4303834201D1012010BD491CC9B2DE
:100A80000629F3D3002010BD4C0C00206801002083
:100A9000EC00030070B5144E4FF48030C6F8080324
:100AA0000025C6F84051114C606810B9104802F09A
:100AB000B5FCA57062680123656073640D48016828
:100AC000001F00681430B1F5804F04D2B0F5404FDC
:100AD00001D9637005E0814201D3012000E00020CC
:100AE0006070BDE870401047008000404001002069
:100AF000E50004004485004001480068004700000C
:100B00003000002002E008C8121F08C1002AFAD1F4
:100B100070477047002001E001C1121F002AFBD17D
:100B20007047022000F0DAB970B50024064D06E0E7
:100B30006868012110F8340006F020F8641C287859
:100B40008442F5D3002070BD38000020F8B515466A
:100B50000C460646052A01D20720F8BD06F006F924
:100B600018B906F0C9F80028F7D1124900224E60E2
:100B70000C708D60C1E90422C1E906220E4D0DE022
:100B800006EBC4002968009181788DF80110007887
:100B90000A4A694606F03EF80028DED1641EE4B237
:100BA000EED2BDE8F84004480021054A001D00F0DF
:100BB00053B80000380000203C7B00008D25000069
:100BC000A124000072B605F035FC00BF05F088FADC
:100BD0000028FBD1104C0121208801EB00400FA11F
:100BE00005F08AFB10480068C00700D000BE2088CE
:100BF000022101EB00400DA105F07EFBBFF34F8FFA
:100C00000948E43801680D4A01F4E06111430160CC
:100C1000BFF34F8F00BFFDE7800100204661746184
:100C20006C206572726F7200F0ED00E0537973749E
:100C3000656D207265736574000000000400FA059C
:100C40000EB500210091CDE901106A4644F2010081
:100C5000FFF7B8FF0EBD0000074B9B7823B12AB108
:100C600020B10068037C1BB1082070470720704743
:100C70004174426100207047FC02002070B506F00C
:100C8000A3FB104800240B21047044700E4D8170AA
:100C900014206C602C706C70FFF7D6FC07211420B8
:100CA000FFF72AFD1420FFF706FD0848046007211E
:100CB0001120FFF721FD0548001F0068A8600020F3
:100CC00070BD0000FC020020580000200815014003
:100CD0002DE9F843DFF8709099F802305BB350B318
:100CE000052902D20720BDE8F88343691BB3437C82
:100CF000012B22D0002704460025884616462846A8
:100D000000F036F8684606F0DFFEC0B10121017040
:100D10000E4944600968C0E90218C0E904769DF8EC
:100D2000000089F80100002000F024F81420FFF7EB
:100D3000D8FC2846D7E70820D5E70F46DBE704258F
:100D4000002000F017F8F4E7FC0200200415014031
:100D50000649897839B130B1416921B10021017466
:100D6000022106F073BC082070470000FC0200203E
:100D700000F002B800F008B872B602480168491CD9
:100D8000016070476C00002003490868401E08603D
:100D900000D162B6704700006C00002070B50546B7
:100DA00008680C46411C04D003F0CFF8206803F01B
:100DB0005DF86068411C02D0002103F045F8296805
:100DC000A069C1F82405607D227D29681043C1F81F
:100DD0006C05D4E900122868C0F81425C0F80C1579
:100DE000207D012814D1A068411C02D0002103F00D
:100DF0002BF8E068411C04D003F0A7F8E06803F08A
:100E000035F8D4E902122868C0F80825C0F8101592
:100E100070BD70B5054608680C46411C04D003F04F
:100E20009EF8206803F02CF86068411C02D0002175
:100E300003F013F82968A069C1F82405607D217DBD
:100E40002A680843C2F86C05D4E900122868C0F883
:100E50000C15C0F81425207D012814D1A068411C70
:100E600002D0002102F0F9FFE068411C04D003F039
:100E700076F8E06803F004F8D4E902122868C0F8B4
:100E80000825C0F8101570BD2DE9FC410646C007C5
:100E90004FF000050ED0104F00240122385D009560
:100EA00000231146019502F059FF641C042CF4D371
:100EB00000F04EF8B0070DD5074E0024361D002275
:100EC000305D032300951146019502F047FF641C35
:100ED000042CF4D3BDE8FC81F87A0000094908B578
:100EE000085C0090684602F0EDFFD0F80425009BF6
:100EF0000121994021EA0203C0F808351140C0F8E9
:100F00000C1508BDF87A00000249085C012103F0C5
:100F100030B80000F87A00000249085C002103F0B4
:100F200028B80000F87A0000084908B5085C00906D
:100F3000684602F0C7FFD0F804050099C84010F0D9
:100F4000010000D0012080F0010008BDF87A000007
:100F500010B500242046FFF7D7FF641C042CF9D3FA
:100F600010BD10B500242046FFF7D6FF641C042CEA
:100F7000F9D310BD10B50246064B4FF0FF300021EB
:100F80005C5C944201D1084610BD491C0429F7D38A
:100F900010BD0000FC7A000070B50023042810D2B8
:100FA0000D4D00EB4004012A02D101290CD0002292
:100FB000094E00EB4000304461B1012906D00229FE
:100FC00006D00723184670BD0E30C2B22A55F9E785
:100FD0004270F7E78270F5E7C401002030B4826800
:100FE0000468531C8360A154D0E901128A4202D3E1
:100FF00030BC02F0BABD30BC7047400003F05CB9B1
:10100000FFFFFFFFFFFFFFFFFFFFFFFFFFFFFFFFF0
:10101000FFFFFFFFFFFFFFFFFFFFFFFFFFFFFFFFE0
:10102000FFFFFFFFFFFFFFFFFFFFFFFFFFFFFFFFD0
:10103000FFFFFFFFFFFFFFFFFFFFFFFFFFFFFFFFC0
:102000002DE9F0470D468146FEF7B4FF044604284B
:1020100036D2DFF874801B481C4EA8F10C0725B39C
:10202000012D0ED0022D2BD104EB44003044457815
:10203000002D25D0B968002922D02846BDE8F047F8
:10204000084704EB4401755C0E44717849B10E4AAF
:102050004FF40041093A8068FEF73AFE08B987F864
:102060000390B17808F80410E2E78068FEF770FE8C
:1020700004EB4401314418F804008D78A842D7D00D
:10208000BDE8F087007B00000C000020C4010020A8
:1020900070B506461E480024C0E90161B00720D58E
:1020A0000025012211462846FEF776FF6D1C0446E6
:1020B000042D02D2002CF4D013E094B940F26662F1
:1020C00004211448FEF742FD04000AD1FEF72CFD5E
:1020D000040006D10F48104A0021001FFEF7BCFD86
:1020E0000446F00712D00120FEF7CEFE74B909486D
:1020F0000A4A00210C38FEF7AFFD040006D105485E
:10210000074A01210838FEF7A7FD0446204670BDA6
:10211000000000200C7B0000792300000D2F000040
:10212000230B00002DE9F05F6A4C0546002660781D
:10213000B34618B184F801B000F0D0FE664F4FF4FA
:102140007A694FF4C87A4FF00108182D62D2DFE89F
:1021500005F0AC0C0C31404D62676B746B74BE7D46
:102160007D7D7D7DACAFB2B5BEBE0020FEF7DCFE4E
:1021700000284FF0000008D0FEF7C6FE022D02D165
:102180004FF4E16008E0484606E0FEF7C5FE022D88
:1021900001D1C82000E05046410CC0034FF4FA7250
:1021A000801841F10001257052000023FEF7B6F8B7
:1021B00001462AE00020FEF7B7FE00284FF000009D
:1021C00004D0FEF7A1FE4FF44870E5E7FEF7A4FE49
:1021D000DFE70020FEF7A8FE00284FF0000002D045
:1021E000FEF792FECFE7FEF797FED4E70020FEF75A
:1021F0009BFE00284FF0000002D0FEF785FE01E0B4
:10220000FEF78AFE257041F69A1100223868FEF723
:102210005FFD064646E00020FEF760FE257008E000
:10222000002051E025703DE084F801800120FEF798
:1022300055FE002240F6CD41E8E784F801800120F8
:10224000FEF74CFE00224FF48041DFE77868FEF78E
:102250007FFD0646D5F1110000D02EB10220FEF719
:1022600053FE84F802B01DE0012816D980B2C821BF
:102270004843C117C90341EA5041C0034FF4FA7201
:10228000801841F1000152000023FEF747F8014693
:1022900000227868FEF71CFD06460220FEF73CFE91
:1022A00084F802803046BDE8F09F00F017FEB9E7E1
:1022B00000F014FEB4E700F011FE04E000F00EFEA2
:1022C0000020FEF729FE0120FEF726FEAAE7FEF712
:1022D00048FEA7E700000020007B00002DE9F04742
:1022E0000546861C90460F464FF001090020FEF778
:1022F0003FFD1B4C20683860D4E90001401AA168FA
:1023000004F21C47081A0EE00121384601F08EF84D
:1023100000F082FE0146384601F088F8D4E9000159
:10232000401AA168081A401C8642EDD8B8F1000F87
:1023300003D0052065F3891002E0062065F39F5065
:10234000A2682168114004EB8101C8602068304414
:1023500020600020FEF70EFD4846BDE8F087000033
:1023600008050020034803C8814201D101207047BD
:10237000002070470805002000780221FFF740BECA
:1023800005494FF0FF32082841F8202002D30844C5
:1023900080F858207047000020020020F0B54FF070
:1023A000FF3512B10023082601E008230C260C4C4F
:1023B00005E000BF54F823707F1C04D05B1CB342BF
:1023C000F8D32846F0BD26185DB286F8305044F8A0
:1023D0002310002AF5D1E11881F85800F1E7000038
:1023E000200200200249084490F9300070470000A4
:1023F000200200202DE9F05F26484168F1B3DFF8A4
:1024000098B00E688146DBF8004087688078E11B51
:1024100021F07F45ED1CB0B9DFF880804FF48030AB
:10242000C8F84403C8F804031120FEF70DF9112081
:10243000FEF741F94FF0010AC8F800A02F2004F080
:1024400095FB89F802A0B54200D23546124BE81937
:102450003C3320F07F401860DBF800105A46091B1F
:1024600021F07F41001B20F07F40C91C81420FD921
:10247000106818602F2004F079FB00E004E0BDE84C
:10248000F05F1120FEF72DB9BDE8F05F04F09CBFAE
:10249000BDE8F09F580000200415014000100140E5
:1024A0002DE9F0470025DFF88C803CE060680021D2
:1024B00000EBC506012032789146FDF760FFD4E9B4
:1024C000062300EA020701EA030C57EA0C0728D0AA
:1024D00082438B434846C4E9062304F005FC327866
:1024E0008246914601200021FDF749FFD4E90423EB
:1024F00000EA020401EA03074A4650460021FDF7BC
:102500003EFF44404F403C430BD17078012801D03E
:10251000012100E00021726881EA0A010AB14846FF
:1025200090476D1CEDB298F8000044468542BDD33B
:10253000BDE8F0873800002010B50021024800F007
:1025400080FF80F3100010BD240900200E4910B553
:102550000A784C780023A24212D0521CD2B20A70E0
:10256000022A00D10B70084A0B780C3252F8232053
:1025700002608868104420F07F408860012010BD10
:102580000360002010BD0000580000202DE9F0413C
:102590008046024601200021FDF7F1FE1A4F054654
:1025A0000E467868FEF7D4FB00280CD1174CD4E90E
:1025B000062110462A4001EA06031A4305D0A84323
:1025C000B143C4E90601BDE8F081404604F08CFB4C
:1025D00030B1D4E9040128433143C4E9040105E0E2
:1025E000D4E90410A943B043C4E90410D4E90601B6
:1025F00028433143C4E90601A1687868BDE8F04189
:102600000022FEF765BB00003C7B00003800002084
:1026100010B501F033FD00BF01F032FE0028FBD100
:1026200010BD10B50024204601F086FD641C082C66
:10263000F9DB10BD10B501F0AFFD012804D0FFF7A4
:10264000E7FF012001F0B6FE01F01AFE002803D1D9
:10265000BDE8104001F020BD10BD10B5002420469B
:1026600001F07AFD641C082CF9DB10BD02490A88D0
:102670000280897881707047947B0000F0B507462E
:10268000204889B0154600780E4698B1012814D02C
:10269000022834D110221C4904A8FDF783FE1B49EF
:1026A0000D2204A8FDF77EFE0024164A6846521C3F
:1026B00021460DE010221449F3E71022124904A824
:1026C000FDF770FE04A800F088F8EDE7052C02D2B3
:1026D000135D035500E00155641CE4B2102CF5D3E2
:1026E00001F026F804A801F035F86946084600F024
:1026F000F5FF2B466A463146384600F01BFB09B011
:10270000F0BD0000E4000020977B00004C09002091
:102710000149087070470000E400002001460D22C6
:102720000148FDF73FBE00004C0900200349026844
:10273000C1F801200079487170470000E4000020D2
:1027400070B5084C0D46E2784AB10749FDF72AFEFC
:102750000DB1E07828700020E070012070BD0020ED
:1027600070BD0000EA000020590900200248C0782E
:10277000002800D001207047EA000020F0B54E2369
:10278000B3FBF2F5022303704F23841804F8013CD5
:1027900081B10123541E0BE003F003068E5DB6FBEE
:1027A000F5F705FB176605FB0366C6545B1CDBB239
:1027B000A342F1DB01210DE04318445C13F8013C16
:1027C000E31ADBB2052B03D2C3F1050323444354C0
:1027D000491CC9B29142EFD3F0BD41F201010A6830
:1027E00002600979017170470349D1F8072002603E
:1027F000C97A017170470000EA000020F8B505466B
:102800004FF480500E468079FF2815D1002141F207
:10281000060003F051FF002441F207070AE00121FE
:10282000684600F00BFA9DF80010E01903F044FF31
:10283000641CE4B2B442F2D3002206E041F2070085
:10284000805C521C05F8010BD2B2B242F6D3F8BD3F
:1028500030B58BB020203E4D00240890AC7020464F
:1028600001F0AEFC002805DD08AA6946002001F051
:102870002DFC0446E87820430AD1012001F0A0FC99
:10288000002805DD08AA6946012001F01FFC044666
:102890003CB39DF8000007283AD2DFE800F0043985
:1028A000080C10233400684600F0B4F830E06846A5
:1028B00000F08CF92CE0684600F04AF928E00A2084
:1028C0008DF8240009AC601CFFF78EFF00F04EF875
:1028D00010B9601CFFF72AFF0122062109A800F0A9
:1028E00087F815E06C460120FFF712FF1022611CEB
:1028F000601CFFF7C3FE601C00F010FA40B1201D01
:10290000FFF70CFF04E00898C1B2684600F0E4F855
:1029100001F0B6FC60B90020FEF76FFB687828B1C3
:1029200001F05AFC40F0010001F05AFDFFF782FE71
:1029300007490020C91D0A5C521C12F0FF020A540C
:1029400003D1401CC0B20528F5D30BB030BD000048
:10295000EA00002000B500F009F8002802D0024982
:102960000220087000BD0000EA0000200248007844
:10297000002800D001207047EA00002008B504219B
:102980006846FFF73BFF684600F074F901F024FC4D
:1029900040F0020001F024FD0449002048708870D6
:1029A0000870C870FEF729FB08BD0000EA0000208F
:1029B00070B50E4D04466878A04216D0FFF728FE89
:1029C00034B101F009FC40F0010001F009FD07E01D
:1029D00001F002FC20F0010001F002FD002028704F
:1029E0006C70BDE87040FFF725BE70BDEA000020A6
:1029F00070B516460C460546FFF70AFEFFF72DFE9A
:102A000022462946304601F0EFFABDE87040FFF754
:102A100011BE0000FEB5054620202E4E029000207B
:102A2000B070FFF7F5FD01F0D7FBC4B2301D90F98F
:102A3000010010F1400F44DB002001F0D1FC962092
:102A4000FEF7DBFAFFF7EDFDFFF7F4FD01F018FCF0
:102A50000028FBD108208DF8000004210DF10100B1
:102A6000FFF7CCFE05226946002001F0BDFA4FF4C5
:102A7000AF70FEF7C2FA012001F0B2FCFFF7DAFDF9
:102A800001270CE0002001F09BFB40B102AA29467F
:102A9000002001F01BFB2878012800D1B77001F05D
:102AA000EFFB0028EED1FFF7D8FDFFF7BAFD0020BD
:102AB000FEF7A3FA204601F093FC00BFFFF7BAFD32
:102AC000FEBD24F0010001F08BFC4FF4FA70FEF71C
:102AD00094FAF3E7EA0000203EB50D460446FFF7FE
:102AE00045FF08B1002000E00220FFF711FE681E3C
:102AF000C2B2611C601CFFF7C1FD601C00F00EF942
:102B000038B111482D1FEAB2C270211D0F48FDF7E0
:102B100049FC0B208DF800006C46A01DFFF7A6FDB8
:102B20000322A11DA01DFFF7A9FD601CFFF75CFE9D
:102B3000FFF71CFF10B9601CFFF7F8FD0122092107
:102B40006846FFF755FF3EBDEA0000205909002006
:102B50003EB50446FFF70AFF002827D00020FFF704
:102B6000D7FD0322611C601CFFF788FD601C00F08C
:102B7000D5F800281AD0144B00246D461878022886
:102B800015D003281AD08DF8044009208DF80000D4
:102B90002C46681CFFF76AFD0922611C601CFFF7C8
:102BA0006DFD01220A216846FFF722FF3EBD01208C
:102BB0008DF80400681DFFF710FE02E002208DF87A
:102BC00004001C70E1E70000EA0000207CB5194D0C
:102BD0000446687800282BD0FFF7C8FE20B9601C97
:102BE000FFF7A4FD012028706846FFF7F6FD0021DD
:102BF0006846425CFF2A02D1491C0529F9DB0529F8
:102C000016D1FFF7F1FD69460523621C084600F066
:102C100091F8094869460078FF2809D1052241F258
:102C2000010003F06BFD00214FF4805003F044FDE0
:102C30007CBD0000EA00002000100000F0B50B4B46
:102C40000025C3F8005101241C602A46084E09E003
:102C5000D3F80071002FFBD037688754C3F80051B8
:102C6000521CD2B28A42F3D35C60F0BD00D0004067
:102C700008D500402DE9FF41054601F001FB264C37
:102C80000646EDB328786978EA7800EB0120A97848
:102C9000090401EB0261471801F0FCFB204601F03A
:102CA00017FB50B10021084601F0F2FA28B138466E
:102CB00001F01EFB08B1012402E0012407E037B156
:102CC0002146084601F0E4FA08B1012700E0002798
:102CD000641CE4B2082CF2D301F052FA0446C2B2EA
:102CE00029466846FFF74AFD87B12146684601F04C
:102CF0000FFB58B10120002E05D001F0CDF900E006
:102D000007E030B1012004B0BDE8F0810020002EC2
:102D1000F9D00020F7E700000406080A10B50322E6
:102D20000349FDF76AFB08B1002010BD012010BD6A
:102D3000947B000070B5002409E000BF11F8015B2E
:102D400012F8016B7540641C00F8015BE4B29C4210
:102D5000F4D370BD0278521C027002788A4201D30B
:102D600000210170704700002DE9FC5F0E008346D2
:102D7000DDE90C47C6F1000098469246814600D432
:102D80000846012503E000BF90FBFAF06D1C50459A
:102D9000FADAA84500D9454624B1002E01DB7807B0
:102DA00000D5641EB80702D5B8F1000F0AD0F807A5
:102DB00008D13CB1A54205D220215846641EFEF739
:102DC0000DF9F6E7002E02DA4E462D2102E07807D3
:102DD00003D52B215846FEF701F907F0030002281E
:102DE0000BD1B8F1000F08D13CB1A54205D230217A
:102DF0005846641EFEF7F2F8F6E7CDE90047434671
:102E000052463146584604F005FEBDE8FC9F0000DE
:102E100070B50D46044600684FF4887103F0A0FEBB
:102E20004FF49071206803F09BFE4FF4927120687C
:102E300003F096FE4FF4A271206803F091FE206823
:102E40001249C0F8041320686907000B40B2090E4C
:102E5000002806DA00F00F0000F1E02080F8141DD1
:102E600003E000F1E02080F8001420680121000B4D
:102E700040B200F01F0291404009800000F1E020C4
:102E8000C0F88012C0F8001170BD000010030200ED
:102E9000024600201268930702D0530702D47047FD
:102EA000500714D502F00300012802D002280CD1EB
:102EB00005E0C2F383100B68801C184404E0022371
:102EC000086803EB925210440860012070470868BC
:102ED00000EB9253C2F38910401CEEE70A4810B58C
:102EE000807860B1002401E0022C06D02046FEF775
:102EF0000BF8641C042CF7D310BD0324F6E7BDE8DF
:102F00001040FEF725B800000000002003480179BA
:102F1000C90702D00078FFF705B97047000000200C
:102F20002DE9F047394E002780463D46DFF8E09016
:102F3000D6F804A057E003D00446D0F81C8035E052
:102F400099F8002002EB4201521CD2B289F800200D
:102F500009EBC10199F80230091D9A4201D189F8A3
:102F6000005048680A780446012A12D0022A02D08A
:102F7000032A3BD108E004F039FB00B10127257496
:102F800034E00574C06900E070680028F9D1706011
:102F90002CE0207C50BB88686060C868A06008692D
:102FA000E0604869A061F07800B165606268B1686E
:102FB000184B501A20F07F40984202D2A168084472
:102FC00006E0881AA16820F07F40814202D9081AE1
:102FD000206000E0256065600120A5602074204627
:102FE000E56104F0E5FAB8F10000A4D199F8001009
:102FF00099F801008142A3D117B97168514502D0F7
:103000000120BDE8F0870020FBE700005800002009
:10301000FC020020FFFF7F002DE9FF41002623482E
:1030200000F001FA2148001F074600F0FCF9204C8F
:1030300060680090A56800E000986946284004EBAD
:1030400080000C30FFF724FF0028F5D101AA009979
:1030500001EA050304EB8303491CDB6842F82030D6
:10306000401C00910228F2D3019800F003000128CF
:103070000BD0022810D10198032101EB9050009948
:10308000BDF80A6001EB900005E00198BDF80A6008
:10309000C0F3831008440090384600F0C1F908B12D
:1030A0000098606004B03046BDE8F081200900203F
:1030B000080500208AB0FDF7E1FD08B1FDF7C0FD6D
:1030C00000210120FEF7E4FF08B1FDF7B9FD4FF440
:1030D0000041002003F06AF908B1FDF7B1FD02F0EC
:1030E000F1FF0120FDF7D0FE012001F085F828B99D
:1030F00001F04CF800F50340FDF7A2FD4FF4FC7021
:1031000001F07EF928B901F041F800F50340FDF720
:1031100097FDFFF733FC01F05FF840F0040001F089
:103120005FF928B901F032F800F50340FDF788FD9A
:103130000120FFF73DFC00F0AFFF28B901F026F8B1
:1031400000F50340FDF77CFD17480321008801EBE3
:10315000004016A103F0D0F802F0C2FF0028FBD116
:103160005FF02004FFF774FBFFF700FC08B1FFF7E6
:10317000F1FB0220089401F023F828B108AA69465F
:10318000022000F0A3FF07E0FFF7F0FA0028E9D0E3
:1031900008A96846FFF7D4FA0028E3D09DF800009C
:1031A00004F032F8DEE700008001002047617A6514
:1031B0006C6C2064796E616D6963207061697269FD
:1031C0006E67206578616D706C65207374617274D0
:1031D00065642E20486F7374206D6F64652E000047
:1031E0002DE9F047C7880446181D16468946B0FBEE
:1031F000F7F1B0FBF7F207FB12009A193A44D21C20
:10320000B2FBF7F2DDF820A001E02468491E002996
:10321000FBD13D1A8846B54216D818E0BAF1000F26
:1032200005D0211809EB08002A46091D04E02044B6
:1032300009EB08012A46001DFDF7B4F800202468B8
:10324000761BA844B74201D9354600E03D46002E22
:10325000E4D1BDE8F087000030B5024659B103F073
:10326000D1F80021074C09E004EB810315685B8865
:10327000AB4202D11160002030BD491C8142F3D322
:10328000052030BD6C0100202DE9F0415C49037838
:103290000446D1E903020025082B77D2DFE803F0CA
:1032A000042B4877726E8795217C914208D238B101
:1032B00000EB81018A6C521C8A640168491C016020
:1032C000A17B2E4661F307062189677B61F31F46C8
:1032D0006189606861F30F05217B61F31745E17B2C
:1032E00061F31F6501F0F6FC2A4631463846BDE819
:1032F000F04100F0C2BE4869407D10B9414800F07D
:103300008DF82F46218965F3070761F31F4761890F
:10331000267B61F30F05617B606861F31F6501F037
:10332000D9FC2A4639463046BDE8F04100F0A4BE3B
:10333000217B914208D238B100EB81018A6C521C8A
:103340008A640168491C0160A07A217A60F307054C
:1033500061F30F25E17A667A676861F3174538B142
:103360001FB92848263000F059F8384601F0B2FC61
:1033700029463046BDE8F04100F030BFBDE8F041DD
:1033800000F088BE00F082FFBDE8F08131E01E4809
:103390004168491C416001780029F5D0816811B16C
:1033A000491E8160F0E7BDE8F04100F067BEA379F7
:1033B000934208D238B100EB830293685B1C9360A0
:1033C0004268521C42608A680CE0A379934208D29A
:1033D00038B100EB830293685B1C93604268521C17
:1033E00042604A68002ACFD061792079BDE8F04177
:1033F0001047BDE8F04103487F3000F00FB80000EF
:10340000FC0000203D0405006809002002490F224D
:103410000A70886170470000FC000020FFF7F6BFCB
:10342000002100F009B8012100F010B808B56A4683
:10343000FCF723FF009808BD08B56A46FCF703FFB8
:1034400008BD08B56A46FCF7E5FE08BD08B56A4642
:10345000FCF7ECFE009808BD08B56A46FCF71AFFB9
:10346000009808BD70B5044600252846FDF780FC8D
:1034700021686268086890420ED9401E0860017891
:10348000A38AE26801FB0325227A2168101AC0B2E0
:103490000A79824200D208710020FDF76BFC2846B1
:1034A00070BD70B505460C460020FDF761FCE8686C
:1034B000A98A201AB0FBF1F12A681068431C136036
:1034C0000170BDE870400020FDF754BC10B530B16C
:1034D000017A42680368891AC9B21A6006E00E20B0
:1034E00010BD03681A68541C1C601170491EC9B2D3
:1034F000F7D2006800210171084610BDC20800F033
:1035000007030120895C98400840704710B5C20845
:1035100000F00703885C01249C402043885410BDC0
:1035200070B5074C251F206829684968884202D376
:103530000448FFF773FF286821688068405C70BD0D
:103540003801002044000100014800687047000075
:103550003801002010B50446054800684068A042C4
:1035600002D80448FFF75AFF0148001D046010BD4F
:10357000340100204C000100014840687047000001
:103580003801002010B50446054800680068A042D4
:1035900002D80448FFF742FF0148001D446010BDF7
:1035A000340100205800010010B5040002D1054884
:1035B000FFF734FF044800210460001D01604160F2
:1035C00010BD000027000100340100200948021F3F
:1035D0004168491C416012681368994208D300236E
:1035E00043600168491C01605268914200D3036046
:1035F0007047000038010020002839D0401E00BF6D
:1036000000BF00BF00BF00BF00BF00BF00BF00BFC2
:1036100000BF00BF00BF00BF00BF00BF00BF00BFB2
:1036200000BF00BF00BF00BF00BF00BF00BF00BFA2
:1036300000BF00BF00BF00BF00BF00BF00BF00BF92
:1036400000BF00BF00BF00BF00BF00BF00BF00BF82
:1036500000BF00BF00BF00BF00BF00BF00BF00BF72
:1036600000BF00BF00BF00BF00BF00BF00BFC5D18B
:1036700070470000F0B505460478154889B0164635
:1036800040F82420124A08690832A2F10C0742F8D7
:103690002400487F385520226846FCF783FE0494B6
:1036A0002878385C48B10EB10A4A00E00022694629
:1036B000281D03F0C5FC09B0F0BD0EB1064A00E0BC
:1036C0000022694605F10C0003F08CFBF3E70000D3
:1036D00014000020F17800003D77000070B5124D15
:1036E00006464FF080746868814202D01022FCF7D1
:1036F00059FE0E490020C1F8000101220A6001E0D4
:10370000641E0ED0D1F80021002AF9D0C1F80001C2
:10371000A9688E4203D010223046FCF743FE0120F8
:1037200070BD002070BD00002400002000E00040BB
:103730000549064801F11002C0E90012103282600A
:103740000348016001207047F001002024000020A0
:1037500004E500400146024810220068FCF722BE42
:10376000240000202DE9F0410446102802D30B4824
:10377000FFF754FE094E0A4D761D204600F07EF8F4
:10378000070008D0AF4202D13046FFF747FE384667
:1037900000F03AF8F1E7BDE8F0810000D000030046
:1037A000ADDEADDE01480068704700006801002012
:1037B00010B50020114A014600EB40039C186170CF
:1037C000A170D154401CC0B21028F5D3DE22CC2108
:1037D0000B48FCF7F9FD0A4A0020A2F1180100BFCE
:1037E00000EB001302EB430341F82030401CC0B251
:1037F0000628F5D303490620086010BD5C0B0020A5
:10380000640C00206801002070B5104C064620684A
:10381000062802D30E48FFF701FE3046FDF710F9E7
:1038200018B90B48401CFFF7F9FD0A4D20680A49FA
:1038300055F82000884203D00548801CFFF7EEFDB4
:10384000216845F82160491C216070BD6801002095
:10385000800003004C0C0020ADDEADDE10B5044648
:10386000102802D30348FFF7D9FD034904EB4400B5
:10387000085C10BDC20003005C0B002070B5002680
:103880000446102802D30C48FFF7C8FD0B4D04EB8B
:103890004404285D70B105F1300000EB840160192B
:1038A00010F8022F51F822600321FFF753FA285D28
:1038B000401E2855304670BDA20003005C0B00205E
:1038C00070B50C460646102902D31248FFF7A6FD34
:1038D0003046FDF7B5F818B90E48401CFFF79EFDBD
:1038E0000D4D04EB4404285D032810D205F130008F
:1038F00000EB8401601910F8012F41F822600321C8
:10390000FFF728FA285D401C2855012070BD0020D3
:1039100070BD00008C0003005C0B002010B5044655
:10392000102802D30948FFF779FD094904EB440048
:103930000A5C42B101F1300202EB80020844807857
:1039400052F8200010BD002010BD0000B30003009D
:103950005C0B00200B4810B50168002479B10A4ABD
:103960000A4B02EB8102491E52F8044D13600160BC
:103970002046FDF765F810B90548FFF74FFD2046D2
:1039800010BD0000680100204C0C0020ADDEADDE53
:103990007800030000487047408100402DE9F74F50
:1039A000904607004FF0000502D13448FFF736FD7E
:1039B000334C4FF4803BC4F808B3324EB07818B1A2
:1039C0002E48801DFFF72AFD706818B12B4809307A
:1039D000FFF724FDDFF8B0A077605FEA08004FF042
:1039E00000094FF00108AAF1040724D001282FD0C4
:1039F000022829D021481D30FFF710FD86F80280EB
:103A0000C4F840910199294489B239603F68C4F8EB
:103A10004480DAF80060D4F8400118B117482B3020
:103A2000FFF7FCFCAF4215D3AE4201D3BE4221D317
:103A3000124833301CE0C4F84480DAF80050C4F86F
:103A40004080C4F84091D9E70F48001D0568D5E7CC
:103A50003D68D3E7BE4201D2012000E00020B5421C
:103A600001D8012100E00021884203D103483E3003
:103A7000FFF7D4FCC4F804B3BDE8FE8F8600040051
:103A8000008000404001002044850040004870470D
:103A90004880004070B5144C01266660E66066649C
:103AA00012480025056011483C30006810B11048EC
:103AB000FFF7B4FC4FF0FF30C4F80803C4F84051DE
:103AC0000A490420083108600A48456006704570BC
:103AD00085700820FCF7CEFD4FF0E0214FF4807098
:103AE000C1F8000170BD0000008000400885004062
:103AF00047000400400100200148007870470000A2
:103B0000400100200349012008600349002008709B
:103B100070470000008000404001002070B5074859
:103B200001250561C560064C0026082066606670A8
:103B3000FCF7A0FDA670257070BD0000008000405D
:103B400040010020014840787047000040010020FB
:103B50000FB408B50399002904D004AA00926A465C
:103B600000F00FF801B05DF814FB10B58268044650
:103B7000002A05D0D4E90403216898470020A060FA
:103B800010BD2DE9FC4791460C00804676D014F814
:103B9000011B39B125290ED04046FDF71FFA2078C8
:103BA0000028F4D198F80C00002867D04046BDE802
:103BB000FC47FFF7DABF0020012221782B291BD018
:103BC0002D2902D0302908D102E040F0010001E0A7
:103BD00040F00200641C002AEFD100252A290ED0F3
:103BE0002178A1F130020A2A11D205EB850201EBFE
:103BF0004205641C303DF1E740F00400EAE7D9F8E3
:103C000000100B1DC9F800300968641C0D442178B0
:103C100000232E290BD114F8011FA1F130020A2A2A
:103C200005D203EB830201EB4203303BF3E76C293F
:103C30000DD068290BD0692921D00BDC252918D09B
:103C4000582931D063290ED0642915D117E014F812
:103C5000011FECE7702969D0732932D075291BD078
:103C6000782909D120E0D9F80000011DC9F8001019
:103C700001784046FDF7B2F9641C90E76CE0D9F892
:103C800000100A1DC9F800200968CDE900500A2279
:103C90004046FFF769F8EFE7D9F800100A1DC9F8A8
:103CA000002009680A2206E0D9F800100A1DC9F8A8
:103CB000002009681022CDE90050404603F0AAFE1A
:103CC000DAE7D9F8001000270A1DC9F800200E68AD
:103CD000C00705D112E04046761C7F1CFDF77EF937
:103CE00031780029F7D104E0202140466D1EFDF710
:103CF00075F9BD42C0D9002DF6D1BDE74EB13046B1
:103D0000FCF774FB074604E0202140466D1EFDF7DA
:103D100065F9BD4206D9002DF6D103E04046761C78
:103D2000FDF75CF931780029F8D1A5E7D9F8000052
:103D3000011DC9F80010056830214046FDF74EF915
:103D400078214046FDF74AF908200021CDE900011D
:103D5000034610222946B0E7BDE8FC872DE9FF4164
:103D60001C46DDE90A7815460E46684600F0AAF8BA
:103D700046EA450141EA840141EA072242EA084154
:103D8000009A00EB8200C0F80017BDE8FF812DE922
:103D9000FF411C46DDE90A7815460E46684600F0EC
:103DA0009FF846EA450141EA840141EA072242EAD6
:103DB0000841009A00EB8200C0F80017BDE8FF81BF
:103DC0002DE9FF411C46DDE90A7815460E46684696
:103DD00000F094F846EA450141EA840141EA0722ED
:103DE00042EA0841009A00EB8200C0F80017BDE8E3
:103DF000FF812DE9FF411C46DDE90A7815460E4694
:103E0000684600F089F846EA450141EA840141EA42
:103E1000072242EA0841009A00EB8200C0F800172E
:103E2000BDE8FF811CB5002100910B4601220191E4
:103E3000FFF7C6FF1CBD1CB5002100910B460122F7
:103E40000191FFF7D6FF1CBD1CB500220B46009266
:103E500011460192FFF7B4FF1CBD1CB500220B46B2
:103E6000009211460192FFF7C4FF1CBD1CB5002152
:103E700000910B46012201911146FFF7A1FF1CBDE5
:103E80001CB5002100910B46012201911146FFF75C
:103E9000B0FF1CBD13B50C46684600F021F8009930
:103EA00000EB8101D1F8002722F44032C1F800274D
:103EB000009900EB8100D0F8001741EA0441C0F8F6
:103EC00000171CBD0168202902D24FF0A0407047A6
:103ED00001F01F010160014870470000000300501D
:103EE0000168202902D24FF0A040704701F01F0165
:103EF000016001487047000000030050016820295C
:103F000002D24FF0A040704701F01F01016001484C
:103F100070470000000300500168202902D24FF0D2
:103F2000A040704701F01F01016001487047000088
:103F30000003005001B56846FFF7D2FFD0F8100526
:103F40000099C84000F0010008BD01B56846FFF7C0
:103F5000D5FF009A01219140C0F8081508BD01B5B0
:103F60006846FFF7D9FF009A01219140C0F8081573
:103F700008BD38B501240090684631B1FFF7A2FFB3
:103F800000998C40C0F8084538BDFFF79BFF0099A9
:103F90008C40C0F80C4538BD1CB5094C0144D4E92F
:103FA0000034CDE900346C4606E000BF54F8203000
:103FB000D3F81035401C08C28142F7D81CBD000060
:103FC0002C7B0000034908B508440021016000680B
:103FD000009008BD0060004002494058012800D010
:103FE00000207047006000402DE9F041204D16464A
:103FF00088460746082801D3042035E0B8F1000FB1
:1040000003D0202E03D906202EE003202CE03846D2
:1040100001F01AFA032801D3092025E0384600F000
:10402000ADFF032801D30A201EE000F0D3FC0228D4
:1040300001D2082018E000F057FE044606704078D0
:10404000324640F0010060704146A01CFCF7AAF91E
:10405000F8B2214601F0FAF910B10120BDE8F08173
:104060000448FFF7DBF90F2028700020F6E7000076
:10407000FC000020FC0005007047704710B500F000
:104080006DFD18B1BDE8104000F004B8BDE8104067
:1040900000F062BC7047000010B50B4C606928B19D
:1040A00000F012FB0004000C02D005E0022008E042
:1040B000002000F023FE18B100F062FC012010BDCA
:1040C00011202070002010BDFC0000202DE9F041DF
:1040D00016460F46044600F051FF154D48B157B142
:1040E000204600F057FF00783168814205D2062053
:1040F0001AE00B2018E0032016E0204600F040FFF5
:1041000004000DD0A01C0BD02278A11C38463260D0
:10411000FCF748F9204600F0DDFD0120BDE8F08104
:104120000448FFF77BF90F2028700020F6E7000015
:10413000FC0000202601050010B5082804D305491D
:1041400004200870002010BDC0B200F00DFF012057
:1041500010BD0000FC000020084910B54A69527DDE
:104160000AB10C2002E0082803D3042008700020C4
:1041700010BDC0B201F050F9012010BDFC000020BC
:104180000148006970470000FC00002001480078E9
:1041900070470000FC00002010B500F0E9FC30B1D1
:1041A000012806D0022806D00448FFF737F902207C
:1041B00010BD002010BD012010BD000097010500BA
:1041C000082804D3034904200870401F704700F0FA
:1041D000D5BE0000FC00002000F0DEBE03B50028C4
:1041E00006D10448BDF8041081809DF80610817145
:1041F0000CBD0000EA0000202DE9F0411D4D0646EF
:1042000000241D482C70AC610460446084601B482D
:1042100000F002FC686140B3042000F073FA05F17D
:104220001C00296900F074F80746304600F0C2F817
:1042300000EA0706002000F0A5F80640012000F083
:10424000EFF80640022000F085F80640002000F05C
:1042500009F90640012000F075FE0020EC6000F036
:1042600033FD16B10120BDE8F08101202870002047
:10427000F9E70000FC0000206809002089320000F6
:1042800001484069407D7047FC00002070470000F5
:10429000084A10B553695B7D0BB1022002E0082883
:1042A00003D304201070002010BD00F037FD012062
:1042B00010BD0000FC0000200449002200280A7004
:1042C00002D0886001200870704700006809002053
:1042D000064910B54A69527D1AB1022008700020C3
:1042E00010BD00F0F7F9012010BD0000FC00002017
:1042F000064910B54A69527D1AB1022008700020A3
:1043000010BD00F0F3F9012010BD0000FC000020FA
:1043100010B50F4C6269527D0AB1022014E01029D9
:104320000FD871B178B10A462161014608481C30A6
:10433000FCF738F8064821691C3000F0F7F9012035
:1043400010BD072000E003202070002010BD0000F9
:10435000FC0000200A4910B54B69024601205B7D34
:104360000BB1022004E0012A05D0022A04D00E205D
:104370000870002010BD002000F056FA012010BD8A
:10438000FC0000200A4910B54B69024600205B7D05
:104390000BB1022003E032B1012A03D00E200870D5
:1043A000002010BD012000F0BBF9012010BD00006D
:1043B000FC00002010B540B1012808D002280BD025
:1043C000064905200870002010BD012000E00220F1
:1043D00000F0D4FB012010BD0020F9E7FC00002014
:1043E000064910B54A69527D1AB1022008700020B2
:1043F00010BD00F0D7FD012010BD0000FC00002022
:10440000064910B54A69527D1AB102200870002091
:1044100010BD00F045FF012010BD0000FC00002091
:10442000014610B50020072914D2DFE801F0040F7F
:1044300006080A0C0E00042008E0FC2006E0F82024
:1044400004E0F42002E0F02000E0EC2001F018F895
:10445000012010BD02490E200870002010BD000090
:10446000FC0000200A4910B54B69024600205B7D24
:104470000BB1022003E032B1012A03D00E200870F4
:10448000002010BD012001F005F8012010BD000042
:10449000FC00002010B5FFF7F3FE002806D0FFF760
:1044A000EDFD30BFFFF7ECFE0028FBD110BD000092
:1044B00010B501F0E1F903490020086102490870D4
:1044C00010BD0000C0090020280100202DE9FE4396
:1044D0004D4800684D4C012802D04D48006828B96D
:1044E00060680078202801D8012100E00021494EB1
:1044F00003204FF0000830704348C4F800800830B3
:104500000568424F183F89B300684149083908607F
:1045100002A8CDE900043C480C300268012329467A
:10452000184602F03DF910B3012805D0022821D029
:10453000032855D0384851E0029818B136481C3845
:10454000FEF76CFF284602F08EFA18B932481B3885
:10455000FEF764FF01F0C4F9B97D0023CDE9000145
:104560007068EAB290F9161018461CE01EE02A485E
:10457000113833E0029818B927480D38FEF74EFF7E
:10458000284602F070FA18B923480C38FEF746FFA7
:1045900001F0A6F9B97DEAB2CDE900017068012306
:1045A00090F91610029800F077FB19E000F06CFE0D
:1045B00030B101F095F90146BA7DE8B200F03EFB5A
:1045C0000023CDF800801A4619461846CDF804801D
:1045D00002F0E6F8042803D00F480F30FEF71EFF64
:1045E000206838B1012060750C48206104203070CB
:1045F000BDE8FE8301F040F984F81580C4F810800E
:1046000000F00EF8F4E7000000140040C00900209C
:10461000341500402801002044060900B946000076
:1046200070B5FFF745FF1F4D012028701E48016837
:104630001E4A21F0FF0112691143016002F01CFAC9
:104640001A4C4C3410B302F017FA032802D0184861
:10465000FEF7E4FE022001F04DFB002001F0A2FB7A
:1046600002F00AFA032803D011480830FEF7D6FEFC
:104670002878012803D00E480E30FEF7CFFE022026
:104680002870002020610B48E06070BD02F000F847
:104690000228DFD302F016F960600028DAD104485E
:1046A000401FD5E728010020301500407409002084
:1046B000F4050900CD440000024905200870FFF709
:1046C000AFBF0000280100200148006A70470000C9
:1046D00074090020034910B5086200F0B3FD0249D7
:1046E000086010BD740900201C150040034910B576
:1046F000486200F0A7FD0249086010BD740900205F
:10470000201500400449487704490A6822F4E02251
:1047100042EA004008607047740900201815004004
:1047200001490876704700007409002070B50C003C
:10473000054602D10748FEF771FE1DB90548401C29
:10474000FEF76CFE0448C0E90145BDE8704000205A
:10475000FEF700BFB3030900D809002010B500F030
:1047600093FD044901F1640208B1C86800E088685B
:10477000106010BD740900201CB510494FF4407042
:10478000086002F079F9012812D0022810D003281D
:1047900013D100200090034602460146019001F02B
:1047A000FFFF042809D0BDE81C400548FEF736BECF
:1047B0000021084602F0A4F8F3E71CBD08F501400B
:1047C00048020900144981F8310014490A6822F0AE
:1047D000FF020A6048B1114A0B1D0832012807D0B8
:1047E00002280ED00E48FEF719BE08680860704710
:1047F000086840F001000860FF20106040F20710D8
:1048000007E0086840F0020008604FF6FF70106093
:1048100004481860704700007409002034150040F7
:104820002E04090021100100044981F832000449D6
:1048300008B1012800D10860704700007409002009
:10484000101500402DE9FF413E480068012802D0C4
:104850003D48006830B93D4840680078202801D8BC
:10486000012700E0002700F0FBFB384C0126183C34
:1048700000B9266102F000F9012802D03448FEF7A1
:10488000CDFD344D6868007D18B13148401CFEF7FD
:10489000C5FD00F0F1FFEFB30121084602F030F84A
:1048A00020B1012828D0022826D10FE001F018F805
:1048B000064601F03DFFC7B201F034FF8446A07DFB
:1048C0000021CDE90260CDE900710DE001F008F8AA
:1048D000804601F02DFFC7B201F024FFA17DCDE994
:1048E0000076CDE90281844668686289218990F961
:1048F0001630604600F0B2F9FEF726FEE06013487D
:104900004C3840696060FFF729FF04B00020BDE823
:10491000F04100E001E0FEF735BE6E7000F0B4FC3F
:1049200000280CD000F0DCFF054601F001FFA27D5D
:1049300004B02946BDE8F041C0B200F07FB9BDE83F
:10494000FF8100000014004034150040C009002021
:10495000370709002801002010B5012080F31088D6
:104960000648417D29B1817819B90121817000F093
:1049700045FB002080F3108810BD0000A80900202E
:1049800070B5124C607D00281ED100F0BDFA04F114
:104990003005A86810B90E48FEF740FD686818B9E0
:1049A0000B48401CFEF73AFD02F096F818B1084893
:1049B000801DFEF733FD002002F0AEF80120607587
:1049C000BDE8704000F01ABB70BD0000A8090020CF
:1049D000CE02090001F0B8BE30B50D4D85B0687D3E
:1049E000002813D000F048FB00F046FF0024AC7014
:1049F0006C7505208DF80000684601F0F5FD05484E
:104A0000047005B0BDE83040FFF7B6BE05B030BD5C
:104A1000A8090020280100202DE9F04105460120C9
:104A200080F31088484E4FF003080024707086F819
:104A30000080B470746034817481F460074634611E
:104A4000347506F118007475046044608460C460B5
:104A500004610475183084604460FFF71BF8284631
:104A600001F0FCFD01F072FE002002F047F806F1B3
:104A70003000FEF799FD00210820FBF74DFE0021D4
:104A80000120FBF749FE01211520FBF745FE01201F
:104A900000F074F8A6F13405FF202861042068773F
:104AA0002A4929622A49696285F82870022185F815
:104AB000291085F82A8085F82B00052085F82C0020
:104AC000062085F82D00072085F82E00082085F89F
:104AD0002F0085F8304085F8311085F83270692054
:104AE00045F8140B1E2028604FF4167045F8100C82
:104AF000022000F085FC0F2000F088FCEC802F7174
:104B00006F712C72204601F019FE7078012802D0D6
:104B10001048FEF783FC3770B47074603481748180
:104B2000F46034610C48347574758460447000F02E
:104B3000EBF90820FBF793FD1520FBF790FD84F3BC
:104B400010880148BDE8F081A809002004070A0D7B
:104B500005080B0E9F020900280100200348407D34
:104B600008B100207047012070470000A80900200C
:104B70000148007870470000A809002010B5012105
:104B800081F3108807490A78824204D04870487D32
:104B900028B100F033FA002080F3108810BD00F037
:104BA00003F8F8E7A809002030B5224D85B0287831
:104BB000697888423BD008B900F0A6F9687808B94E
:104BC000FFF7DAFD1C480024046000F055FE194888
:104BD00018300460446004618460C460287801284F
:104BE00002D0022808D015E001F046FF90B1002164
:104BF000084601F085FE0DE0FFF75AFC01F03CFF8E
:104C0000032807D1002300941A4619461846019438
:104C100001F0C6FDFFF7A2FD6878287004208DF82A
:104C20000000684601F0E0FC012005B030BD002026
:104C3000FBE70000A809002054F5014000B585B04D
:104C400006238DF806208DF805108DF804008DF8E8
:104C50000030684601F0C8FC05B000BDF0B585B075
:104C60000DF1280C9CE8F0008DF80C308DF80D400B
:104C70004FF0000C0190ADF808108DF80E508DF833
:104C800000C0ADF80A208DF80F608DF810706846EE
:104C900001F0AAFC05B0F0BD70B586B00226DDE9D2
:104CA0000A458DF808108DF8092001908DF80A301A
:104CB0008DF800608DF80C508DF80B40684601F0BF
:104CC00093FC06B070BD0000014988607047000089
:104CD0002801002010B5012181F3108801F05CFD4E
:104CE000002080F3108810BD10B5012080F31088DB
:104CF00001F054FD002181F3108810BD10B5044669
:104D0000082802D30348FEF789FB0348204490F8A3
:104D1000280010BDAD0309007409002070B50828F3
:104D200019D20F4A024482F828108207D40EFF22BB
:104D3000A240D243042801D20A4D01E0094D2D1DA5
:104D4000286810402860084600F06AFA2968A040E8
:104D50000843286070BDBDE870400348FEF75EBBA5
:104D60007409002024150040A703090010B51B4C4E
:104D700000206070FEF7D4FB19490860FEF7E4FBE1
:104D80001849887501F078FE012807D001F074FEFB
:104D9000022802D01448FEF741FB002000F0AAFFD1
:104DA000FEF7F8FD114908606068091D4068086059
:104DB000A068002811D0007820B1FEF7EBFDA168B3
:104DC00000F0F6FBA0680179002906D000F0C4FBD2
:104DD000A068BDE8104000F0CDBB10BD2801002048
:104DE00008150040A80900209706090050F5014069
:104DF00010B501F0EBFD002820D011480021018101
:104E0000418101F095FC0F49086001F091FC0121FE
:104E100081400C48001D026822F0FF02114301602E
:104E200001F080FC064C1834206001F075FC6060D5
:104E30000548E060BDE81040FFF798BF10BD0000D6
:104E4000A80900202C150040454800001548002105
:104E50000160012101601448016821F48071016042
:104E6000016821F00F01891D0160016821F47021A2
:104E700041F440310160001D016821F000710160C2
:104E8000016841F080710160016821F0FF0141F08B
:104E900020010160016821F47F4101600120FBF7DE
:104EA000DEBB0000FC1F00401415004070B5134C21
:104EB0001348A16800F08AFE6060114C4C3C607F92
:104EC000FFF720FC206AFFF705FC606AFFF70EFC85
:104ED0000025601990F828102846FFF71FFF6D1C69
:104EE000082DF6D3074914F8300F08606078FFF7F3
:104EF00069FCA078BDE87040FFF796BC280100204F
:104F0000C00900200C1500400C4910B500200860B5
:104F10000A484FF440744C380460FFF797FFFEF7DF
:104F2000B5FD064908310860091F054808600348B7
:104F300050380460BDE81040FFF7B8BF54F5014099
:104F40000411004010B504460448406810B90448F4
:104F5000FEF764FA0348047510BD00002801002024
:104F60006E040900C009002010B5012181F31088EA
:104F700001F076FD002080F3108810BD01F073BDB4
:104F800010B5012181F3108801F070FD002181F33B
:104F9000108810BD01F06DBD014800697047000028
:104FA000740900200149086170470000740900205D
:104FB00003490122086101460248FEF7EFBC0000E8
:104FC000A8090020E56A000070B50C4601F0A4FDB8
:104FD000074D2869A04202D30648FEF71FFA286948
:104FE0000122211A0448FEF7D9FC0020286170BD77
:104FF000A8090020D6060900E56A000010B5FEF7F2
:105000007BFD012822D101F081FD10B11048FEF78F
:1050100005FA002264210F48FEF7C0FC0E48007F0D
:1050200080B90E480121016000220007C0F800216C
:10503000016000BF00BF00BFAFF30080D0F80011D7
:105040000029FBD0BDE81040FEF75CBD10BD00009C
:10505000B4060900E56A0000740900201405004048
:10506000044810B5006918B9FEF76CFD002800D09F
:10507000012010BDA809002010B5FEF73DFD012854
:105080000ED0FEF74BFD0748007F10B901208107C5
:105090004860002001F040FD0249002034314860A2
:1050A00010BD0000740900200B4810B54068407D19
:1050B00030B1012000F076FE08490889401C0881C3
:1050C0000749002008600548343803C8BDE810408F
:1050D000091A0020FFF778BF28010020A809002046
:1050E00054F5014070B586B0FFF7BAFF494D4A4EFE
:1050F00005F1340458B100F0BDF8A078002869D05B
:10510000FEF764FA06B0BDE87040FFF765BC207892
:10511000012802D0022804D008E000F0FFFE28B1E8
:1051200070E0307804286DD003286BD0FEF74EFA7B
:1051300000F0A0F8A07868B1FFF74EFC01F0A8FAE3
:10514000022840D303208DF80000684601F04CFA95
:1051500006B070BDFFF728FD20B100206968FFF799
:1051600033FFEBE72078F0B1012816D0022817D0E2
:105170002A48FEF753F9687E0128DFD100F084F851
:105180000028DBD12078D8B1012811D00228D5D051
:1051900022481A30FEF742F9D0E700F087F8EAE734
:1051A00000F008F9E7E700206968FFF70DFFE2E784
:1051B00001F062FC0028C1D101F0DCFB0028BDD168
:1051C000FFF75AFFBAE706B01448BDE87040363022
:1051D000FEF724B92078022808D0FEF7F7F96968AD
:1051E00006B00020BDE87040FFF7EEBE307804281E
:1051F00008D0032806D0FEF7E9F906B0BDE87040F4
:1052000000F0D8B8686806B04008BDE87040FFF705
:10521000CFBE00007409002028010020D00409003E
:10522000024610B50020014622FA01F303F0010303
:10523000C1F10704A3400343491CC9B2D8B20829ED
:10524000F2D310BD2DE9F04100240646254618276B
:10525000E80026FA00F0C0B2FFF7E2FF694207EB70
:10526000C101884020436D1CEDB20446042DEFD3EC
:10527000BDE8F0810348416809B1491E4160FFF76C
:105280006DBA0000A809002004480178022902D064
:105290004068002800D0012070470000A8090020C5
:1052A0000149486070470000740900202DE9F04171
:1052B00086B000F0E1FA01F0DFFB3A4D05F134046D
:1052C00020B3688BB0B3218981423BD301210020F8
:1052D00001F016FB01F026FA26898046648901F068
:1052E00027FA074600F0FCFA014601208DF800007D
:1052F000ADF808608DF80C70CDF80480ADF80A4068
:105300008DF80D10684601F06FF944E001F0C0F926
:10531000022840D3FFF7B8FF68B1FEF72DF9D0BBE4
:10532000287E20B9FEF710F9E168884233D1FFF7F3
:105330005FFD30E006E0E068FEF70CF90020FEF7C4
:1053400021F9F4E7FEF7FEFB10B11748FEF766F807
:10535000FEF7E6F815490968884202D06089401CCA
:10536000608113484078A0B9FFF78EFF88B101F043
:10537000DFF9064600F0B4FAA17D8DF806108DF82D
:10538000050007228DF800208DF80460684601F0C2
:105390002BF9FFF7EBFC296806B00120BDE8F041CE
:1053A000FFF712BE740900207C05090008150040B3
:1053B0002801002070B50024FEF7B2F80D4D2968D1
:1053C000884207D0FEF7ACF82860FEF7BDF80A491E
:1053D000012488750948641E0078044201D1FFF752
:1053E0001FF9054834384168BDE870400020FFF7D8
:1053F000EBBD000008150040A8090020280100208E
:105400000149C860FFF7AAB9740900200149886002
:10541000FFF7A4B97409002010B50446012181F3F7
:1054200010880748017821B1407D10B10548FDF78B
:10543000F5FF204601F026FB002080F3108810BD08
:10544000A80900206803090001F025BB10B501225E
:1054500082F3108801F02CFB58B10848817819B903
:10546000407D08B1FFF7CAFD002080F310880120BD
:1054700010BD002080F3108810BD0000A809002096
:10548000024981F830000249086070477409002021
:105490000C1500400149087770470000740900208E
:1054A00070B51149114A0025487802EB0010027BC3
:1054B00022B10F4AD2F80C2102B10125807A08707E
:1054C000012000F0DFFB0B4C1DB1A068806800B12B
:1054D00080476068002806D00179002903D0BDE824
:1054E000704000F01BB870BDE4090020A87B0000EC
:1054F000001000404801002007480069012805D03D
:10550000022805D0032805D100F09AB800F04CB964
:1055100000F0E4B870470000E4090020827B00211D
:1055200093000B4A1344C3F81019C37B02EB8302A8
:10553000C2F81019427B0121837BC07B01FA02F281
:1055400001FA03F3814003481A430A43026070479B
:1055500000F0014008F501404279054BC079012176
:1055600003EB80000AB101667047016370470000D9
:105570000060004082680021C2F84011C17B094AE6
:10558000CB0009490B44C3F81025C37B826801EBAB
:10559000C301C1F81425C17B01208840034908607C
:1055A000704700001011004000F0014004F5014078
:1055B0002DE9F0410746886800260C46C0F8406196
:1055C0008868097B1A4D00F5A07005EBC101C1F890
:1055D00010056278E178207B00F08EFC607B05EBA3
:1055E000C000C0F81075617BA06805EBC101C1F86F
:1055F00014051048C0F80C61C0F81061A17B0E487A
:1056000005EBC101C1F810056278E178A07B00F0DC
:1056100061FC217B0120627B00FA01F100FA02F2B9
:105620001143A27B9040014304480160BDE8F08132
:1056300000F00140001000400C11004004F5014052
:105640002DE9F0411F4E02200025307003207070BC
:1056500075603575B0691C4C401CB061C4F80C51C4
:10566000C4F80051C4F81051C4F80451C4F82851CA
:10567000C4F80052681EC4F808030120FBF705F8BF
:10568000124FB868007D50B1114800684042B075B3
:10569000C4F81C510120A0610E49800208600C482A
:1056A00044380068F168884202D00B48FDF7B6FE26
:1056B000B868C068002802D0BDE8F0410047BDE8E6
:1056C000F0810000E40900200010004048010020A3
:1056D0004815004008F5014051040A0010B52D4C52
:1056E000D4F80C01012802D02B48FDF797FED4F81E
:1056F0001001012803D02848401CFDF78FFED4F884
:105700000001012803D02448801CFDF787FED4F84F
:10571000040118B12048C01CFDF780FE0020C4F829
:105720000C01C4F81001C4F80001C4F80401C4F865
:1057300008010221C4F800120121C4F8081308224C
:10574000C4F80423154A0323154C137010755060D8
:10575000606890B1027912B1FFF7E0FE0DE00278C7
:105760005AB1027B437B807B01FA02F201FA03F318
:1057700081400C481A430A430260A068006900B1E6
:105780008047A0688068002802D0BDE8104000472C
:1057900010BD000000100040F3030A00E4090020DF
:1057A0004801002008F501402DE9F0412A4DD5F8C7
:1057B0000001012802D02948FDF730FED5F8040188
:1057C000012803D02548401CFDF728FE2448016825
:1057D000244801700021C5F80011C5F80411C5F86E
:1057E0000811491EC5F808130126C5F8046381682D
:1057F0001D4F097D09B1B1023960446814B32079A5
:1058000000B3617BDFF86480A06808EBC10100F59C
:10581000A070C1F810056279E179607B00F06CFB43
:10582000607B06FA00F03860207B114908EBC0006D
:10583000C0F810156279E179207B00F04BFB207BEA
:1058400086403E600B480649091FC06808600B206F
:10585000C5F80002BDE8F08100100040BD030A0059
:10586000081500404801002004F5014000F0014007
:105870000C110040E409002070B50120FAF710FF78
:105880000120FAF702FF144C4FF0FF30C4F8080370
:105890000026C4F80062C4F8106101202061A061F4
:1058A0000E4D2878012813D0022813D0032811D0D8
:1058B0005FF00100FDF7A0FEC4F810612E706E7558
:1058C000002000F0DFF9BDE870400120FAF7FEBECD
:1058D0000620EFE70220EDE700100040E409002079
:1058E00001480078704700004801002001F03F01A6
:1058F0004FF4003343EA0121830009481844C0F8FB
:105900001015D0F810150AB941F48011C0F810151F
:10591000D0F8101541F00301C0F8101570470000D1
:105920000060004008480069012806D0022806D01F
:10593000032806D00548FDF771BD00F095B800F0CA
:1059400007B800F0F1B80000E409002033050A00B0
:105950002DE9F047DFF8F0800421012088F80010DD
:10596000D8F81810491CC8F81810FAF78EFE3748F6
:105970000068374D2870374C0026C4F80C61C4F815
:105980000061C4F81061C4F80461A868DFF8C89029
:105990000127007DA0B1304808380068400502D4D6
:1059A0002E48FDF73BFD294840300068404288F80A
:1059B0001600C4F81C61A7614FF48061C9F800109B
:1059C000D4F8000118B125480930FDF727FDD4F8B7
:1059D0000C0118B121480A30FDF720FD4FF0E020FE
:1059E000B046D0F8000210F0020F03D01B480B3075
:1059F000FDF714FD6E68CEB13078B8B1C4F80C81F3
:105A0000717B184A164802EBC101C1F81005727883
:105A1000F178707B00F05EFA707B0F4907FA00F0B6
:105A2000091F0860F07B8740C9F80070A868C0684B
:105A300000B18047A868417D002903D00349006870
:105A4000091F0860BDE8F087E40900200815004040
:105A5000480100200010004008F50140C0040A0081
:105A60000C11004000F001402DE9F041294C0026C6
:105A7000C4F80C61C4F80061C4F81061C4F808618E
:105A8000C4F80461012004F58074FAF7FEFD0820D3
:105A9000C4F804020125C4F808520720C4F8000124
:105AA0001D484468002C32D0207920B1207B1B494E
:105AB00005FA00F008602078002828D0A068C0F817
:105AC0004061A17B164FA06807EBC10100F5A070F3
:105AD000C1F810056278E178A07B00F00DFAA068AB
:105AE000C0F84061E17B0F4807EBC101C1F8100528
:105AF000E17BA06807EBC101C1F81405A17B05FAA1
:105B000001F0E17B8D4005492843091F0860BDE88D
:105B1000F0810000001000404801002008F501401D
:105B200000F001400C11004070B5234CD4F80C017A
:105B3000012802D02148FDF771FCD4F8100101289A
:105B400003D01E48401CFDF769FCD4F80001012871
:105B500003D01A48801CFDF761FC0020C4F80C013A
:105B6000C4F81001C4F80001C4F80401411EC4F8CF
:105B70000813C4F80002124C626872B1117861B166
:105B8000557B012303FA05F1957BD27B03FA05F5DA
:105B900093400C4A2943194311600B4903220870B2
:105BA0004A7048600875A0680069002802D0BDE806
:105BB0007040004770BD000000100040F5040A006E
:105BC0004801002008F50140E409002070B50646B0
:105BD0000C460120FAF764FDFFF74EFE244D2548E0
:105BE0002649C5E901460024047003264670446036
:105BF00004610475447584751F4808601E48F030C0
:105C0000091F08601E48016821F0010141F0807100
:105C100001600120FAF75AFD686838B3017909B9C3
:105C2000017819B38168C1F808650422C1F810250C
:105C3000027CC2F18102C1F8402540F20112C1F894
:105C40000022C1F804450122CA60C1F8404101792F
:105C500021B142798179C079FFF748FE68680178FF
:105C600021B142788178C078FFF740FE014870BDCD
:105C700048010020E40900201410004064F50140B0
:105C8000741700402DE9F041174C00250746C4F871
:105C90000052164E307803281CD0681EC4F8080342
:105CA000C4F80C51032070700120FAF7EEFC00BF1D
:105CB000C4F80051C4F81051C4F80451756035752A
:105CC000002F0FD00A488068006900280AD0BDE87C
:105CD000F04100476FF00800C4F808030820C4F83A
:105CE0000403E5E7BDE8F08100100040E40900206E
:105CF000480100202DE9F0470746DFF89080224850
:105D00004FF0FF3100EB0716C8F808130120FAF72F
:105D1000BCFC1F4C0025DFF87C9065756770D9F8D6
:105D20000800032F0268A2604168C4E90315A56159
:105D30003068606019D2337AC8F80032C8F80C5164
:105D4000C8F81051F37A14481BB10160006828B1FB
:105D500008E00260006828B9104801E00F48401DC3
:105D6000FDF75CFB717AC8F80413D9F80800007DD0
:105D700028B1022F03D10A49A575780208600120D5
:105D80006075BDE8F0870000A87B000000100040AF
:105D9000E409002048010020041500409C020A008C
:105DA00004F501402DE9F05F404C8246404866789A
:105DB00000EB0617607D012802D03E48FDF72EFB60
:105DC000207D18B13B48401CFDF728FB0125002130
:105DD0002575DFF8E490A0466175032E47D2BAF12D
:105DE000000F3CD1D9F80440BCB32279AAB38A464B
:105DF0000846A168C1F84001217BDFF8C0B0A06867
:105E00000BEBC10100F5A070C1F810056279E179D2
:105E1000207B00F071F82A49C1F80CA1607B294968
:105E20000BEBC000C0F810156279E179607B00F0DF
:105E300051F8217B627B05FA01F005FA02F1084373
:105E400021490860D9F80400204A81791268CA40C3
:105E500012F0010F01D18068056038680560022EDC
:105E600001D0012E07D1B97A88F8001003E011485B
:105E70002530FDF7D3FAD9F80800007D002813D0AB
:105E8000022E11D110480068400503D409482A3079
:105E9000FDF7C4FA0E480068002805D1BDE8F05FA0
:105EA00004482B30FDF7BABABDE8F09FE4090020A2
:105EB000A87B0000B8020A004801002000F0014061
:105EC000001000400C11004004F501401005005086
:105ED00004150040064B03EBC0000AB1054A01E07F
:105EE000044A303A02EB8101C0F8141570470000F3
:105EF00000F0014060600040064B03EBC0000AB1B7
:105F0000054A01E0044A303202EB8101C0F8141561
:105F10007047000000F00140306000400348D0F8B6
:105F20000401012800D0002070470000001000404C
:105F300030B5124B01460020D3F81044224609E048
:105F4000157A854205D1401C0A28F7DB4FF0FF3057
:105F500030BD5268002AF3D1421CF9D00872D3F840
:105F600010242AB152684A60D3F81024516030BD21
:105F70000022C3F810144A6030BD0000080500205C
:105F8000F0B595B01C4615460F4608461A9E00F01F
:105F900009FB182109A8FAF71EFA0E96CDE9095453
:105FA0000023082203A9384600F011FB059806904B
:105FB000BDF81000ADF81C00BDF81200ADF81E00D1
:105FC00000208DF821000398082600F00300012826
:105FD00002D0022818D032E003983346850AC0F375
:105FE000C2008DF8200003980FA9C0F38314A2000B
:105FF000384600F0ECFA09A8009006AB22460FA93B
:10600000284600F02BFA1AE00398840DC0F3C20072
:106010008DF82000082C01D2254600E008253346E3
:106020002A460FA9384600F0D2FA2E44641B09AB69
:1060300006AA29460FA800F063F9002CEAD13846D9
:1060400000F0B6FA15B0F0BD7047012001F094BB26
:10605000084810B50178084A515C19B1001D01F0DB
:106060007BF802E00C3000F089FFBDE81040002012
:1060700001F082BB740000201000002008B5034A24
:1060800000924023024AFFF77BFF08BD65740000C1
:10609000080400200A4A012902EBC00007D00229A7
:1060A00007D0032907D0042907D000207047022019
:1060B00070470420704700797047407970470000AE
:1060C0001C7D000010B5FFF7C0FF04210348FFF757
:1060D0002FFF02490120487210BD000088000020F7
:1060E0002DE9F0478CB0FCF73DF918B100200CB059
:1060F000BDE8F087784C0020C4F81804BFF34F8F38
:1061000060680290A5684FF00008284004EB80000A
:1061100008E021680298814201D86160E6E72840E2
:1061200004EB80000C3002A9FCF7B2FE0028F0D18D
:1061300003AB029901EA050204EB8202491CD26812
:1061400043F82020401C02910228F2D3039800F06B
:106150000300022802D001284ED0A5E00398502267
:10616000810D8946B2EB905F00D850210E4666F350
:106170009F5003900831594800F0CBF9070078D0C0
:1061800000F010FA4346082203A9384600F025FA29
:10619000029908F1080A2940681A8000001D864209
:1061A00023D94D4D0C3530B1C2B204EB8101301A08
:1061B00090460C3104E02946F2B20025904628466C
:1061C000C6B25346384600F008FA0AEB08032DB170
:1061D000324629464FEA070000F0FFF9029909F11B
:1061E000030001EB900002903AE004EB810153467A
:1061F000324638460C31EFE70398C0F38311062985
:1062000000D3062161F389100390C0F38310801C32
:106210008100324800F07DF9070045D000F0C2F956
:106220004346082203A9384600F0D7F908F10808C8
:1062300000260FE00298434600EA0501401C04EBEB
:1062400081010290042238460C3100F0C6F908F1B1
:106250000408761C0398C0F38310B042EAD847B113
:10626000D4F81054D4F8180468B1384600F0A0F9F6
:106270002CE019E0687A012804D12A6828463946BA
:10628000126890476D68002DF4D1384600F090F9FF
:106290000020FAF76DFDD4F8180408B90298606080
:1062A0000020FAF767FD11E0D4F8104404E02168FB
:1062B0002046896888476468002CF8D10848022184
:1062C000008801EB004007A100F016F8FCF74AF83F
:1062D00080F001000BE70000080500204C7D000065
:1062E000800100204261636B656E647320666C758B
:1062F000736865640000000000231A4601F0D2B8FC
:106300002DE9F0470E4680461C46924608293ED8A5
:1063100094F80C90002020731946104600F0FCFF02
:106320000025B54206D218F805201AA12046FDF72F
:106330000FFC03E019A12046FDF70AFC6D1C082D97
:10634000EFD317A12046FDF703FC0025B54210D27C
:1063500018F80570FAF722F80068C05D10F03E0FDB
:1063600001D03A4600E02E220EA12046FDF7F0FBB8
:1063700003E00DA12046FDF7EBFB6D1C082DE5D3D6
:1063800001222146504600F0A9FF84F80C90BDE898
:10639000F087000020253032780000002020200007
:1063A0007C0000002563000020000000104810B5AC
:1063B000FF218160002101604160C0F81814C0F81D
:1063C000141480F820140B4800F0F0F800280DD1C8
:1063D00009480A490A4B401AC108002003E000BFDF
:1063E00023F82000401C8842FAD3002010BD000092
:1063F000080500204C7D00004C7D00001C7D000045
:106400006C01002002480349401AC0087047000090
:106410004C7D00001C7D000013B56846FCF71CFF96
:1064200008B100201CBD0248009950F831001CBD85
:106430001C7D000070B508480125D0F8104480F894
:10644000205405E0657221682046496888476468E1
:10645000002CF7D170BD0000080500202DE9FF4792
:1064600081460C9D00200C462F7B287398461646CB
:106470002946184600F050FF072E42D2DFE806F00A
:1064800004090F161F2A360049462846FDF760FB0F
:1064900037E0494628462268FDF75AFB31E0D4E947
:1064A000002349462846FDF753FB2AE0A0680090E8
:1064B000D4E9002349462846FDF74AFB21E0D4E908
:1064C0000201CDE90001D4E9002349462846FDF741
:1064D0003FFB16E004F1080007C88DE80700D4E987
:1064E000002349462846FDF733FB0AE004F1080083
:1064F0000FC88DE80F00D4E9002349462846FDF770
:1065000027FB00222946404600F0E8FE2F73BDE835
:10651000FF872DE9F041858A80462D1F4819C01C50
:10652000B0FBF5F0C6B24046FCF79CFF041E19D044
:106530000020207101206071E58000272546761E2D
:10654000C4F800800BE04046FCF78CFF60B1617935
:10655000491C6171286005467F1CC0F80080B74265
:10656000F1D32046BDE8F081204600F002F800207B
:10657000F8E72DE9F041457901466B1E002201E064
:106580000968521C9A42FBD30F680146002605E0B9
:1065900038460C68FCF785FF2146761CAE42F7D3DF
:1065A000BDE8F0810121001DFCF740BFFCF78EBF64
:1065B00010B504460121001DFCF74EFF10F0FF0F3F
:1065C00004D12046BDE81040FFF7D3BF10BD38B559
:1065D00001240094FCF704FE38BD38B50024009473
:1065E000FCF7FEFD38BD000070B51A4C054620686A
:1065F00010B91948FCF712FFD4F8D4000A2803D3C5
:106600001548401CFCF70AFFD4F8CC0000EB8000D2
:1066100004EB800115F8040B08712DCD8860CA6069
:106620000B614D61D4F8D400401CC4F8D400D4F8F8
:10663000CC00401CC4F8CC00D4F8CC1000200A29AF
:1066400001D3C4F8CC004FF0E0214FF40010C1F8A2
:10665000000270BD000A00204A000B0010B50400C3
:1066600002D10948FCF7DAFE084941F8CC4B00207A
:1066700041F874098867C8674FF0E0214FF40010B3
:10668000C1F8000110BD00003E000B00000A002010
:1066900010B5074CD4F8D4000A2802D90548FCF7F5
:1066A000BDFED4F8D400C0F10A00C0B210BD000095
:1066B000000A002079000B0010B500F0030290439F
:1066C000D200FF24944003689140A343CA180949AB
:1066D00001230B60BFF36F8FBFF34F8F026006483B
:1066E0000268002AFCD000200860BFF36F8FBFF360
:1066F0004F8F10BD04E5014000E40140F0B51546A0
:106700000E460746002404E0315D3819FFF7D4FF38
:10671000641CAC42F8D3F0BD0148C068704700006B
:10672000D80A00200148806870470000D80A00207D
:106730000148406870470000D80A0020014981F8EC
:1067400081007047D80A0020FDF72CB870B5FDF71E
:106750002FF800240E4E2546204600F067FD04F178
:10676000080000F063FD3555641C082CF4D309487B
:106770000121057045608560C5600561456180F84F
:10678000805080F85850C56780F8811070BD0000B7
:1067900054010020D80A0020FDF736B8FDF7DAB81A
:1067A0002DE9FF4F81B0444FDDE90EA803260025F7
:1067B000F86F0C46AB4610B94048FCF72FFE38780E
:1067C000032803D03D48401CFCF728FEF86FB9466B
:1067D0004178C8072FD199F8810060B3002701984C
:1067E000E8B3039A584662F31700C1F3410161F31D
:1067F0001F6009EB84018A6BCAF800B0C8F800B0CA
:106800000090904234D0204600F050FD051E07EA6B
:1068100005072DD004F1080109EB8102009991616F
:1068200004990D4223D0264E305D00B3204600F07F
:1068300032F910B105E00127D1E720482830FCF7F4
:10684000EDFD204600F029F9CAF80000BAF1000F6A
:106850000AD018B919482E30FCF7E0FD00E01BE023
:1068600006F804B0022603E014483230F4E70126AB
:1068700077B1204600F02DF9C8F8000018B1104893
:106880000121015506E00C485830C8F8000001E02D
:10689000C8F800B00DB107E004264C46D9F87C00DA
:1068A000FCF7B2FFC4F87CB089F800B000F068F8DB
:1068B00005B03046BDE8F08FD80A00202D010C004D
:1068C0005401002010B50C4C207810B10B48FCF797
:1068D000A5FD00F0DFFC00280DD0FF2202704178FA
:1068E00041F00601417000214318491C9A7020298B
:1068F000FAD30321217010BDD80A002007010C0033
:1069000070B51A4C05460E462078012804D002289E
:1069100002D01748FCF782FDB5B12078012803D0DA
:106920001348401DFCF77AFDE06818B91048801D37
:10693000FCF774FDE068007820B1606800F0B6FCF8
:10694000022502E0002500E004254EB1606800F059
:10695000A4F8A168814203D005481D30FCF75EFD14
:106960000020207000F00CF8284670BDD80A0020E6
:10697000CC000C00014890F880007047D80A002035
:106980002DE9F041104C207800281AD194F88000AD
:10699000002816D10825012600276069FCF75EFF54
:1069A00018B184F88060606920616069401C606192
:1069B000082800D1676194F88000002801D16D1E7D
:1069C000EBD1BDE8F0810000D80A002070B5224C60
:1069D000207810B12148FCF721FD94F880000025B3
:1069E000F8B12069606000F074F8A06018B91B4825
:1069F000C01DFCF713FDA0684078C00705D194F8CE
:106A0000810010B10220E56009E0606800F02BF819
:106A1000032806D200F03EFCE06010B10120207097
:106A200002E02078002815D0A06818B90B48203063
:106A3000FCF7F4FC2069606004EB8000C17E491C17
:106A4000C17684F88050C27EA068417862F342012A
:106A50004170012070BD0000D80A002098000C0091
:106A60000830FCF77FBE0830FCF7F8BE0830FCF7B2
:106A700005BF0830FCF752BF01480078704700009E
:106A8000D80A002010B5044600F0F0FB2046BDE80F
:106A90001040FCF767BEFCF7E1BE70B50446FCF79A
:106AA000EDFE050002D0204600F0E0FB284670BD58
:106AB00070B50E4604460025FCF774FE38B1214639
:106AC0003046FCF7FDFE10B1FFF75AFF01252846BE
:106AD00070BDFCF723BF000001480078704700003C
:106AE0005C01002004480178817041780170001D2C
:106AF00050F82100004700005C0100200249887026
:106B000048700870704700005C0100200148407820
:106B1000704700005C01002010B50446022802D333
:106B20000248FCF77BFC0248447010BD33000D00A6
:106B30005C0100204058002800D00120704708B5B3
:106B4000002242504058009008BDD0F8040308408D
:106B500000D0012070474058002800D00120704725
:106B600008B5002242504058009008BD002802D0CD
:106B70000149800108477047517B00002DE9F04131
:106B80000E46804600F05AFB204D0028404616D0A5
:106B9000FBF728FC284490F858008009032802D00D
:106BA00001280AD003E04046FDF7C4F928B10321CB
:106BB0004046BDE8F041FDF76DB90221F8E700F06D
:106BC00049FB002820D04046FBF70CFC0446104F40
:106BD0004FF4807007EB840100EB8400D1F810259E
:106BE00080B242F00102C1F81025FDF7EBF9002E4A
:106BF0000AD04046FBF7F6FB55F82000002803D0EA
:106C00000120A040C7F80403BDE8F0812002002065
:106C1000006000402DE9FC41DFF8C080044608EB2D
:106C20000400002790F930001346C0170E46401CA0
:106C300001D008274FE0B0781946C0F34002204643
:106C4000FBF7ACFB0546401C44D0B07841071CD490
:106C5000C0070DD068460094FDF742F9009900EB9B
:106C60008100D0F8001721F00201C0F8001707E0FA
:106C700000217378204600910A460191FDF787F8BC
:106C8000164920466431FCF741FCB078800718D5DE
:106C90001348317800EB8500D0F81025114B1A40CD
:106CA000C0F810254FF47C524FF4403302EA04221E
:106CB00003EA01410A43D0F810150A43C0F8102531
:106CC00009E008EB0500327810F8581F41EA8211FC
:106CD000017000E004273846BDE8FC812002002056
:106CE00000600040FFC0FCFF10B5FDF723F900284D
:106CF00000D0012010BD000070B5194D95F86A0054
:106D000008B1082070BD0020411E2A18401CC0B2E6
:106D100082F830103028F8D300242046FBF730FBEF
:106D2000641CE4B20C2CF8D30D490024E0204C661E
:106D3000A1F868400B4981F8000401264020891F12
:106D4000C1F88002C1F800014FF4BE70FDF73AF9B6
:106D50000549F007C1F8040385F86A60204670BD54
:106D60002002002006E000E000600040034890F8A8
:106D70006A00002800D00120704700002002002097
:106D80000121B1EB507F01D10120704700207047F5
:106D900070B50D4600F00CFB04000FD00020F9F791
:106DA000E7FF207920B10020F9F7E4FF112070BD42
:106DB0000120256020710020F9F7DCFF002070BD64
:106DC00010B500F0F5FA002802D000210160017131
:106DD00010BD00000149024800F0F6BC8C02002002
:106DE000002000402DE9F0410546007916460F4687
:106DF00000EB40012D4A01EBC00102EB810494F845
:106E00002A1011B10820BDE8F081294951F820105D
:106E10002868FFF7BDFF08B11120F4E7394628467E
:106E2000F9F7BCFF66603869206030004FF001065A
:106E30002FD03F7F4FF48E712868FFF780FE4FF40C
:106E4000A2712868FFF77BFE28681A49C0F804136E
:106E500028684FEA4711000B40B2002806DA00F01C
:106E60000F0000F1E02080F8141D03E000F1E020A5
:106E700080F800142868000B40B200F01F0206FAE8
:106E800002F14009800000F1E020C0F88012C0F853
:106E9000001128680421C0F800150020A061E061FD
:106EA00084F8290044F8140FA675ACE78C02002082
:106EB000347B0000800002002DE9F0470546007990
:106EC0000B4600EB400101EBC000234901EB8004BD
:106ED000284600F043F810B11120BDE8F0874FF0CC
:106EE0000008C4F82080A360626184F828804FF411
:106EF0008E76474631462868FFF721FE28684FF016
:106F00000109C0F808902146286800F0F9FB606884
:106F100000BBD5F800A00EE094F8280008B10F27B8
:106F200016E031465046FFF705FE0028F4D0214612
:106F3000504600F0E5FB216A60698142F1D3314699
:106F40002868FFF7F7FD0028F9D02868C0F80C90F2
:106F5000C4F814803846C0E78C020020007900EBAA
:106F6000400101EBC000044901EB800040690028AA
:106F700000D00120704700008C0200202DE9F0476E
:106F8000044600794FF0000900EB400101EBC0001E
:106F9000254901EB80072068C0F80095786880B12A
:106FA00020682249C0F8081320680121000B40B274
:106FB00000F01F0291404009800000F1E020C0F87D
:106FC00080112068D0F80C25D0F81485D0F8086519
:106FD000D0F810554FF0FF31C0F81415C0F80C155B
:106FE0002068C0F80815C0F81015501C02D01046D3
:106FF000FCF718FFB8F1FF3F02D04046FCF712FF44
:10700000681C02D02846FCF70DFF701C02D03046E9
:10701000FCF708FF2068FFF7D3FE87F82A90C7F82F
:107020000490BDE8F08700008C020020840202007A
:107030000149024800F074BCB80200200020004062
:107040002DE9F0410546164600790F46154A00EB3A
:10705000C00102EB810494F8201011B10820BDE8B2
:10706000F081114951F820102868FFF791FE08B10E
:107070001120F4E739462846F9F7CBFE66603869F7
:1070800020601EB1397F2846FBF7C2FE2868082120
:10709000C0F800150020A061E0610121606184F862
:1070A0002010DCE7B8020020387B00002DE9F04713
:1070B00004460E460079204900EBC00001EB800534
:1070C00017463046FFF75CFE30B1204600F036F838
:1070D00020B11120BDE8F0871020FBE76F61AE60A2
:1070E0004FF49076002731462068FFF739FD4FF4C2
:1070F000AC7841462068FFF733FD2068AA686969CB
:10710000C0F84425C0F848152068012181606868EE
:1071100078B9B14649462068FFF71DFD064641464D
:107120002068FFF718FD0643F4D000B10F270020B8
:1071300068613846CEE70000B802002000790549B2
:1071400000EBC00001EB80004069002800D0012066
:1071500070470000B80200202DE9F047044600798E
:10716000274900EBC00001EB800720684FF00009C1
:10717000C0F80095786880B120682249C0F80813EB
:1071800020680121000B40B200F01F02914040092D
:10719000800000F1E020C0F880112068D0F80C25B4
:1071A000D0F81485D0F80865D0F810554FF0FF31AD
:1071B000C0F80C15C0F814152068C0F80815C0F800
:1071C0001015501C02D01046FCF735FEB8F1FF3FF9
:1071D00002D04046FCF72FFE681C02D02846FCF780
:1071E0002AFE701C02D03046FCF725FE2068FFF70F
:1071F000E7FD87F82090C7F80490BDE8F08700000D
:10720000B80200201003020070B5002405460126D4
:1072100006FA04F02842204602D0F9F77DFE01E08C
:10722000F9F772FE641C042CF2D370BD024A0021EF
:1072300002EB800081617047D80A002004490844AD
:1072400090F93000082801DB0120704700207047CA
:10725000200200200449084490F93000082801D297
:1072600001207047002070472002002010B504461E
:10727000064890F8801021B10069A04201D1FFF7C3
:107280007FFB03490020085510BD0000D80A0020EC
:107290005401002010B5044CE06F002802D1FCF727
:1072A00059FBE06710BD0000D80A002070B5094DF9
:1072B0000446E86F10B90848FCF7B0F804F108017B
:1072C000E86FFCF7FDFA002802D00020E8670120F3
:1072D00070BD0000D80A00202E020C0010B50C462C
:1072E000017A052908D0407A38B1084808A1026817
:1072F0002046FCF72DFC00E01AB106A12046FCF761
:1073000027FC2046BDE81040FCF72FBCC000002041
:10731000257300000D0A000038B5C3880D460446E9
:1073200033B114A0009015A216A12846FCF710FC5A
:10733000217A05291CD0607A48B1A088FEF7AAFE00
:10734000164951F8202016A12846FCF701FCA08818
:107350000021FFF761F803461049207A143951F8EB
:10736000202001B02846BDE830400EA1FCF7F0BB5C
:1073700038BD00001B5B306D000000001B5B313B23
:1073800033316D0025734C6F67732064726F7070BA
:107390006564202825642925730D0A00C00000209B
:1073A000257300003C25733E2025733A2000000021
:1073B0000349884201D1034870470020704700000C
:1073C000002000403000002070B5012670044FF00E
:1073D000E0210025C1F88001084C4010C4F84803A2
:1073E000C4F8080366602F20FFF7C0FBA660044CBA
:1073F0002F20A560FFF7BAFBA57070BD00100140FB
:107400005800002070B5054688690C4600284FF4E6
:10741000847128460AD0FFF792FBD5F81805626AF6
:10742000E1688854606A401C606270BDFFF787FBAA
:10743000D5F8180570BD1FB501238DF80030CDE9D2
:107440000121D0E90012684690471FBD1FB50123F6
:107450008DF800308DF808100192D0E900126846CE
:1074600090471FBD70B50D4C0020D2B22070201D7A
:107470000B4D0378EB5C1BB1001DFFF717FE02E01C
:107480000C30FFF719FD08B1F9F7DAFB6078002836
:1074900002D021780029FAD070BD000070000020D1
:1074A000100000202DE9F84F204D924689460646EF
:1074B0009846012269461846AF68FAF70FFF58B39D
:1074C000009800210446801C09E000BF00EA070381
:1074D0005AF8212005EB8303401C491CDA60414522
:1074E000F4D34FEA164AFBF727F84AEA0041601C3A
:1074F000384005EB80003C4005EB8402C160D06859
:1075000066F3C50068F3891069F39F2020F003003B
:10751000401C20F00400D06095F8200402E000BF79
:10752000FEF7DEFD0028FBD1BDE8F88F080500203E
:107530002DE9F84F1D4C00256846D4E901A6FBF75C
:1075400005F8002738B30023009A61681CE0D1F8E1
:1075500000C00846944503D9ACEB02020A6015E06E
:10756000A2EB0C0263440760D0F80CC0C1698146ED
:10757000BCF1000F08D006EB030828F07F48C0E9F3
:10758000018CC9F81C5005460029E0D128466160ED
:10759000FBF7C6FC03E02846FBF7C2FC10B15046DF
:1075A000FAF728FFE770BDE8F88F000058000020C8
:1075B0000D4B10B5596831B102680C68A24204D86D
:1075C000A21A0A60C161586010BD0B4603E00B4669
:1075D000C969121B21B10C689442F8D3A41A0C603B
:1075E0000260C161D86110BD580000202DE9F04152
:1075F000144E77683D462C4603E0844204D025466D
:10760000E469002CF9D11BE0D4B1A5420BD1F86993
:10761000706040B90C49012088600021B160F070B1
:107620002F20FFF7A3FA2168E069E86110B1026832
:10763000114401607068874202D00120BDE8F081EA
:107640000020FBE75800002000100140F8B5064676
:1076500000240D462046F9F78BFB684600F034FA0B
:1076600068B10570084946609DF800004870002028
:10767000F9F780FB1420F9F734F82046F8BD04240C
:107680000020F9F777FBF8E7FC0200202DE9F04134
:10769000194D6C68002C2CD0184800270068A96888
:1076A000B846401A20F07F462068B0420CD82146E8
:1076B000361A0744E469087C20B181F81080886993
:1076C00049698847002CEFD129786878814206D132
:1076D000401CC0B26870022801D185F801800648BC
:1076E00069780C3040F82170BDE8F0411420F8F7BB
:1076F000F8BFBDE8F08100005800002004150140EB
:1077000070B50C4605464FF48E71FFF718FA216AE2
:10771000A068415C206A401C2062C5F81C1570BD41
:107720001FB500228DF8002002918168019142610D
:10773000D0E90012684690471FBD00001FB50A46F9
:1077400001788DF8001041680191017A8DF80810D8
:10775000C0680390044850F82210083850F82220DE
:10776000684690471FBD00001C0000200149012011
:10777000087070477000002010B588B004462022C1
:107780000E496846F8F70EFE06200090C01F0190D3
:10779000029003904FF0EB7006900CB1084A00E0A5
:1077A000002269460748FBF765FF08B1F9F748FA78
:1077B0000448001F447008B010BD0000747B000036
:1077C0006D770000740000202DE9FF470C46054648
:1077D0004FF40071FFF7B9F901274FF40178002643
:1077E00018B34FF4927949462846FFF7A3F9E0B160
:1077F00049462846FFF7A3F9C5F8088394F82900FD
:1078000000B96F6002208DF80000D5F88004C5F83B
:1078100080040390A0690290E0680190A661E6618F
:10782000D4E900126846904728E004212846FFF773
:107830008CF918B34FF484712846FFF77BF9E8B14F
:1078400021462846FFF7DEFD616AA069884215D10E
:10785000E06938B1E268616AA0612069E661666248
:10786000E06008E094F8290000B96F60C5F808836B
:10787000A661E268616A2046FFF7DDFD4FF48E786D
:1078800041462846FFF756F978B1206A6169884277
:1078900002D294F8280020B341462846FFF74FF95A
:1078A000616911B12046FFF73BFF4FF4A2784146D2
:1078B0002846FFF73FF9002818D041462846FFF731
:1078C0003EF994F8290000B12F60A06900280DD07E
:1078D000A661E268616A04B02046BDE8F047FFF7A0
:1078E000AABD21462846FFF70BFFDEE7BDE8FF876C
:1078F0001FB50A4601788DF8001041680191017AA0
:107900008DF80810C0680390044850F82210083819
:1079100050F82220684690471FBD00001C00002040
:107920002DE9FF410C464FF4927705463946FFF7A3
:1079300012F90026C0B139462846FFF711F9022096
:107940008DF80000D5F88004C5F880040390D5F8C0
:107950003C058DF80800E0680190A661E661D4E975
:1079600000126846904723E04FF48877394628464E
:10797000FFF7F1F8E0B139462846FFF7F1F8D5F8FE
:107980003C15A069884213D1E06960B1E268D5F87E
:10799000000220F02000C5F80002E069A061206923
:1079A000E661E06001E0A661E2682046FFF74EFD77
:1079B0004FF4A27739462846FFF7CDF860B1394633
:1079C0002846FFF7CDF8A06930B1A661D5F83C157F
:1079D0002046E268FFF73AFD4FF490773946284693
:1079E000FFF7B9F8002813D039462846FFF7B8F852
:1079F000606900280CD0D5F84C058DF800608DF832
:107A00000800A06801906661D4E9001268469047BA
:107A1000BDE8FF812DE9F05F8346DDE90A4A99461A
:107A200090460D460846012703E000BFB0FBF8F082
:107A30007F1C4045FAD2B94500D94F465FEACA706B
:107A400012D18CB15FEA8A7002D5B9F1000F01D072
:107A5000202607E0302605E031465846641EF9F737
:107A6000BDFA0CB1A742F7D35FF00106B9F1010FDF
:107A700002D9A9F1010903E0B5FBF6F0404502D3B4
:107A800006FB08F6F2E7DFF83C9000BFB5FBF6F026
:107A900000FB165519F800105846F9F79FFAB6FB87
:107AA000F8F6002EF2D15FEACA7009D0002C07D098
:107AB000A74205D220215846641EF9F78FFAF5E750
:107AC000BDE8F09F567B00000A494A788B78521C2B
:107AD000D2B2934200D100220B78934201D1002010
:107AE00070470270487800EB400001EBC000001DB9
:107AF00070470000FC0200200D0E0F100B0C18192F
:107B000084010020A4010020D00100200B0003000C
:107B1000012000000C0003000120000018000300F9
:107B200001200000190003000120000000000050A7
:107B300000030050D56D000031700000030000000C
:107B4000DC02002000000000000000000000000037
:107B50000338FDD870473031323334353637383951
:107B600041424344454600007D60000051600000F2
:107B700049600000FFFFFFFFFFFFFFFFFFFFFFFF68
:107B8000FFFFFFFF00000000000000000000D60122
:107B90000701000032536601172D391A440C400DBD
:107BA000490D3E1A2D0C4D000010004010110040F0
:107BB0000310000001000000001000400000000061
:107BC0000B02040000000000041000400000000050
:107BD00007010301000000000040404040404040D9
:107BE0004040414141414140404040404040404090
:107BF0004040404040404040400502020202020234
:107C00000202020202020202022020202020202082
:107C10002020200202020202020290909090909096
:107C20001010101010101010101010101010101054
:107C300010101010020202020202888888888888C8
:107C400008080808080808080808080808080808B4
:107C5000080808080202020240000000D97B000068
:107C60007761726E696E6700646562756700000017
:107C70001B5B313B33306D001B5B306D000000003F
:107C80001B5B313B33316D001B5B313B33326D008D
:107C90001B5B313B33336D001B5B313B33346D0079
:107CA0001B5B313B33356D001B5B313B33366D0065
:107CB0001B5B313B33376D00696E666F000000005F
:107CC0006572726F720000004750494F54450000C2
:107CD0005052530055415254000000005541525437
:107CE0004500000062616C6C6F632E6C6F675F6DA6
:107CF000656D706F6F6C000061707000647D0000D6
:107D0000000000208401000058040000B07D000045
:107D100084010020AC2B0000140B0000C87C000084
:107D200000000000D07C000000000000D47C0000B7
:107D300000000000DC7C000000000000E47C00008B
:107D400000000003F87C0000000003039C000020FA
:107D5000940000209C000020480400207C010020AA
:107D600018000000017A64200040542000400327DE
:107D7000687B33C07C33607C33B87C33687C337879
:107D80007C33707C33807C33887C33907C33987C6C
:107D900033A07C33A87C0318B07C041190D003C2BC
:107DA00005064404192A3F4D33E550031FA950002E
:0400000500000201F4
:00000001FF
